:020000040000FA
:10000000786C0120590200007D0200007F02000090
:1000100081020000830200008502000087020000C8
:1000200087020000870200008702000087020000AC
:1000300087020000870200000F0300005D440000FB
:10004000550700005F070000690700007307000004
:100050007D070000750A00007F0A00009909000072
:100060009F0800000D090000170900002109000089
:100070002B0900003F090000B1060000BB0600008C
:10008000C5060000CF060000E30A0000D509000005
:10009000DF090000E9090000F3090000FD09000084
:1000A000070A0000930600009D060000A706000056
:1000B000C109000041070000870700009107000008
:1000C0009B070000890A0000A3090000110A000034
:1000D0001B0A0000A90800000B070000150700001C
:1000E0003707000095080000D90A00003509000014
:1000F000CF0A0000C50A0000D9060000E306000090
:10010000ED060000F70600002D070000A50700001F
:10011000AF070000B9070000AD090000B7090000F3
:10012000930A00009D0A0000A70A0000B10A00001F
:10013000BB0A0000B3080000BD080000250A00004B
:100140002F0A0000390A0000430A00004B07000094
:10015000710900007B090000C7080000D1080000F9
:10016000C3070000CD07000085090000CB0900008F
:10017000D7070000E1070000EB070000F5070000CB
:10018000FF07000009080000130800001D08000018
:1001900027080000310800003B0800004508000067
:1001A0004F08000059080000630800006D080000B7
:1001B00077080000810800008F0900000107000097
:1001C0001F070000030900004D0A0000570A000045
:1001D000610A00006B0A0000DB080000E50800006F
:1001E0004909000089060000530900005D0900006C
:1001F00067090000EF080000F90800008B08000004
:10020000DFF80CD000F01CF900480047256400001E
:10021000786C0120EFF3108072B67047EFF3108016
:100220007047EFF3108062B6704730BF704780F3BD
:1002300011887047EFF31180704700000138FDD13D
:100240007047000080F30888704780F30988704782
:1002500080F3148870470000DFF83000016841F433
:1002600070010160BFF34F8FDFF82400016821F0B7
:1002700040410160BFF36F8F06480047FEE7FEE78D
:10028000FEE7FEE7FEE7FEE7FEE7000088ED00E0A0
:1002900034EF00E001020000EFF3098141B1F1EE1B
:1002A000101A40F8041D20ED200A29490A68106040
:1002B0007047B0EC200A02C8E1EE101A25490A681E
:1002C00010607047EFF3108072B6704780F31088AB
:1002D000704721484FF0FF010170002080F309882A
:1002E0001E48016881F308881D48012101701D48DE
:1002F0004FF08051016062B6FEE71A484FF080511E
:100300000160704717484FF080510160704772B626
:10031000EFF3098028B1203880E8F00F0C49096814
:10032000086000B5104880475DF804EB0F4810499D
:100330000A780270064807490A680260106890E867
:10034000F00F203080F309884EF0F40E62B670474B
:10035000340000203C00002022ED00E000000020DE
:100360002E00002004ED00E02940000023000020C2
:100370002400002072B6704762B67047EFF3108019
:1003800072B6704780F31088704730BF704720BF47
:100390007047B0FA80F0704790FAA0F0B0FA80F0A1
:1003A000704790FAA0F0704740EA01039B0703D022
:1003B00009E008C9121F08C0042AFAD203E011F8A4
:1003C000013B00F8013B521EF9D27047D2B201E066
:1003D00000F8012B491EFBD270470022F6E710B54A
:1003E00013460A4604461946FFF7F0FF204610BDA3
:1003F000421E12F8013F002BFBD111F8013B02F81D
:10040000013B002BF9D1704710B5002200E0521CCF
:10041000835C8C5CA34201D1002BF8D1D8B2E1B24D
:10042000401A10BD30B504460020034600E05B1CB6
:10043000934203D2E05CCD5C401BF8D030BD00009D
:10044000064C074D06E0E06840F0010394E8070021
:1004500098471034AC42F6D3FFF7D6FE7CB70000C5
:100460009CB7000070B58C1810F8015B15F00703FD
:1004700001D110F8013B2A1106D110F8012B03E03D
:1004800010F8016B01F8016B5B1EF9D12B0705D445
:100490000023521E0DD401F8013BFAE710F8013B8E
:1004A000CB1A921C03E013F8015B01F8015B521EAA
:1004B000F9D5A142D8D3002070BD000000B585B0A9
:1004C000032000214FF400720E4BCDE90132CDE93B
:1004D0000310052003460C4A00900C4803F09AFADA
:1004E000032000214FF40072094BCDE90132CDE920
:1004F000031006200346074A0090074803F08AFAD3
:1005000005B000BD74370120703F0120C54E0000CA
:10051000743F012070470120E34E000086B000F0D8
:1005200083F800F00BFB04464FF47A70B4FBF0F54F
:10053000284603F0A7FF00F0BBFB03F03FFA02F0F0
:100540006BFD02F055FD04F005FD2E4908600846DC
:100550000068012813D142F2107004F0B4FC4FF48B
:10056000803004F0BFFC02F043FD022004F0FEFCEA
:100570004FF4FA6004F0A7FC04F082FC16E0214876
:100580000068022812D142F2107004F09CFC4FF473
:10059000902004F0A7FC02F02BFD012004F0E6FC03
:1005A0004FF4FA6004F08FFC04F06AFC164803C8AC
:1005B000CDE90001154800680590154800680490D1
:1005C000144800680390DDE9041204F0E5FC04F02F
:1005D00073FBFFF773FF13E0012002F0C3FC01205F
:1005E00002F0D2FC4FF47A7003F022FD002002F0FA
:1005F000B9FC002002F0C8FC4FF47A7003F018FD3B
:10060000EAE7000088010020800100207801002036
:1006100074010020700100207047704770477047D8
:10062000704770477047704710B500F05FFA00F0F0
:10063000DFFA10BD10B50446702C04D204F110018D
:10064000C8B200F03BFB10BD70B50446002600BFE9
:1006500000BFFFF793FE064600BF00BF02F046FE54
:1006600000BF00BF3046FFF78DFE00BF00BF702CFB
:1006700004D2044850F8245005B1A84702F050FEB7
:1006800070BD0000EC2B002010B56920FFF7DCFFE7
:1006900010BD10B51920FFF7D7FF10BD10B51A20F7
:1006A000FFF7D2FF10BD10B51B20FFF7CDFF10BD27
:1006B00010B50E20FFF7C8FF10BD10B50F20FFF7D3
:1006C000C3FF10BD10B51020FFF7BEFF10BD10B561
:1006D0001120FFF7B9FF10BD10B52E20FFF7B4FFB2
:1006E00010BD10B52F20FFF7AFFF10BD10B53020A3
:1006F000FFF7AAFF10BD10B53120FFF7A5FF10BD11
:1007000010B55F20FFF7A0FF10BD10B52620FFF742
:100710009BFF10BD10B52720FFF796FF10BD10B549
:100720006020FFF791FF10BD00BFFEE710B532203B
:10073000FFF78AFF10BD10B52820FFF785FF10BD19
:1007400010B51D20FFF780FF10BD10B54320FFF747
:100750007BFF10BD10B50020FFF776FF10BD10B570
:100760000120FFF771FF10BD10B50220FFF76CFFED
:1007700010BD10B50320FFF767FF10BD10B50420B2
:10078000FFF762FF10BD10B51E20FFF75DFF10BD23
:1007900010B51F20FFF758FF10BD10B52020FFF740
:1007A00053FF10BD10B53320FFF74EFF10BD10B53D
:1007B0003420FFF749FF10BD10B53520FFF744FF87
:1007C00010BD10B54820FFF73FFF10BD10B5492000
:1007D000FFF73AFF10BD10B54C20FFF735FF10BDF5
:1007E00010B54D20FFF730FF10BD10B54E20FFF7BC
:1007F0002BFF10BD10B54F20FFF726FF10BD10B521
:100800005020FFF721FF10BD10B55120FFF71CFF4E
:1008100010BD10B55220FFF717FF10BD10B55320C3
:10082000FFF712FF10BD10B55420FFF70DFF10BDEC
:1008300010B55520FFF708FF10BD10B55620FFF783
:1008400003FF10BD10B55720FFF7FEFE10BD10B519
:100850005820FFF7F9FE10BD10B55920FFF7F4FE40
:1008600010BD10B55A20FFF7EFFE10BD10B55B208C
:10087000FFF7EAFE10BD10B55C20FFF7E5FE10BDE6
:1008800010B55D20FFF7E0FE10BD10B56F20FFF73B
:10089000DBFE10BD10B52920FFF7D6FE10BD10B548
:1008A0000820FFF7D1FE10BD10B52520FFF7CCFEC4
:1008B00010BD10B53D20FFF7C7FE10BD10B53E209E
:1008C000FFF7C2FE10BD10B54620FFF7BDFE10BDFC
:1008D00010B54720FFF7B8FE10BD10B56620FFF732
:1008E000B3FE10BD10B56720FFF7AEFE10BD10B50A
:1008F0006D20FFF7A9FE10BD10B56E20FFF7A4FE16
:1009000010BD10B56120FFF79FFE10BD10B5092086
:10091000FFF79AFE10BD10B50A20FFF795FE10BD37
:1009200010B50B20FFF790FE10BD10B50C20FFF79F
:100930008BFE10BD10B52B20FFF786FE10BD10B545
:100940000D20FFF781FE10BD10B56820FFF77CFE7B
:1009500010BD10B56A20FFF777FE10BD10B56B20F3
:10096000FFF772FE10BD10B56C20FFF76DFE10BDD5
:1009700010B54420FFF768FE10BD10B54520FFF705
:1009800063FE10BD10B54A20FFF75EFE10BD10B526
:100990005E20FFF759FE10BD10B50720FFF754FE8B
:1009A00010BD10B52220FFF74FFE10BD10B5362048
:1009B000FFF74AFE10BD10B53720FFF745FE10BD0A
:1009C00010B51C20FFF740FE10BD10B54B20FFF7FF
:1009D0003BFE10BD10B51320FFF736FE10BD10B55D
:1009E0001420FFF731FE10BD10B51520FFF72CFEC7
:1009F00010BD10B51620FFF727FE10BD10B517204B
:100A0000FFF722FE10BD10B51820FFF71DFE10BD28
:100A100010B52320FFF718FE10BD10B52420FFF7F6
:100A200013FE10BD10B53F20FFF70EFE10BD10B530
:100A30004020FFF709FE10BD10B54120FFF704FE6E
:100A400010BD10B54220FFF7FFFD10BD10B56220AC
:100A5000FFF7FAFD10BD10B56320FFF7F5FD10BDDF
:100A600010B56420FFF7F0FD10BD10B56520FFF74D
:100A7000EBFD10BD10B50520FFF7E6FD10BD10B56C
:100A80000620FFF7E1FD10BD10B52120FFF7DCFDCA
:100A900010BD10B53820FFF7D7FD10BD10B53920B7
:100AA000FFF7D2FD10BD10B53A20FFF7CDFD10BD08
:100AB00010B53B20FFF7C8FD10BD10B53C20FFF777
:100AC000C3FD10BD10B52D20FFF7BEFD10BD10B544
:100AD0002C20FFF7B9FD10BD10B52A20FFF7B4FD9B
:100AE00010BD10B51220FFF7AFFD10BD10B50024EA
:100AF00004E0E0B2034900F007F8641C702CF8D35E
:100B000010BD00002907000070B504460D46002600
:100B1000702C10D200BF00BFFFF730FC064600BFAC
:100B200000BF054840F8245000BF00BF3046FFF723
:100B300029FC00BF00BF70BDEC2B00202DE9F04365
:100B4000DFF89CC0DCF8B0C0CCF3007CBCF1000F37
:100B50003ED0DFF88CC0DCF860C1CCF38A26DFF829
:100B600080C0DCF860C1CCF30A0303EB9622DFF807
:100B700070C0DCF864C1CCF30424DFF864C0DCF896
:100B800064C10CF01F05DFF858C0DCF8B0C0CCF32E
:100B9000036111B1032904D101E0124902E01249B5
:100BA00000E000BF00BF01FB02F804F1010C05F1F9
:100BB00001090CFB09FCB8FBFCF0DFF824C0DCF8F1
:100BC000B0C0CCF3090C0CF10107B0FBF7F000E06A
:100BD0000020DFF818C0CCF80000BDE8F08300006A
:100BE00000E00F400024F40040787D0174000020F4
:100BF0002948C06F20F01C002749C8670846C06F0D
:100C000040F01000C8672448C030006823490840FD
:100C10002149C1F8C0002048C0300068204908437D
:100C20001D49C031086048061B49B03108604FF0CB
:100C30004C70086060201B49086004201649C1F808
:100C400064011848A0380068144908401249C1F8E6
:100C5000C0001448A0380068134908430E49C1F881
:100C6000C0000846D0F8600140F40000C1F86001FF
:100C700000BF0C480830006800F0010080F001005F
:100C80000028F6D10448B0300068084908430249FA
:100C9000C1F8B0007047000000E00F4010FC10FCED
:100CA0008100010060E10F40850185010300009093
:100CB00010B500F0F9F800F0BFF810BD2DE9F041D3
:100CC00004464FF00008102C6BD2DFE804F0080E49
:100CD0000F1014293E090A0B0C11120D135300BFFB
:100CE00000BF00BF00BF00BF89E000BF00BF00BF62
:100CF00000BF00BF83E000BF00BFFFF73FFB80469F
:100D000000BF00BF3F48006840F480303D490860A4
:100D100000BF00BF4046FFF735FB00BF00BF6EE0DD
:100D200000BF00BFFFF72AFB804600BF00BF354869
:100D3000006840F400303349086000BF00BF4046FF
:100D4000FFF720FB00BF00BF59E000BF00BFFFF767
:100D500015FB804600BF00BF2A48006840F4802091
:100D60002849086000BF00BF4046FFF70BFB00BFEB
:100D700000BF44E000BF00BFFFF700FB804600BF9C
:100D800000BF4FF0E020006940F001004FF0E0218B
:100D9000086100BF00BF4046FFF7F4FA00BF00BF84
:100DA0002DE04FF0E0204068401C102101EB401086
:100DB000C7B2BC4222DAA4F11000C11700EBD16126
:100DC000C1F34715C11700EBD1614911A0EB4111E7
:100DD000CEB200BF00BFFFF7D1FA804600BF00BF10
:100DE0000120B040A90001F1E021C1F8000100BFDD
:100DF00000BF4046FFF7C6FA00BF00BF00BF00BFFC
:100E0000BDE8F08124ED00E010B5002400BF00BF74
:100E1000FFF7B4FA044600BF00BF1021054802F0F6
:100E2000F1F800BF00BF2046FFF7ACFA00BF00BFDB
:100E300010BD0000DC2B002010B5FFF7E5FF10BD52
:100E40002DE9F04105460C46002714B900BF00F01B
:100E500029F81DB90A202080BDE8F081102128461C
:100E600003F075FF0646102E15D200BF00BFFFF736
:100E700085FA074600BF00BF10222946084803F044
:100E800043FF00BF00BF3846FFF77CFA00BF00BF3A
:100E90000020208002E04FF47A70208000BFDBE762
:100EA000DC2B002000BFFEE710B5002002490860DF
:100EB00000F00AF810BD0000700000200149086031
:100EC000704700007000002010B50A48006840F02C
:100ED000807008490860002007494860084600689B
:100EE00040F001000860FFF729FE04462046FFF7A6
:100EF000E5FF10BDFCED00E0001000E010B50220A1
:100F0000FFF79CF904F0F2F80B48C46904F00C00F8
:100F100008B1022010BD094803F07AFF0220FFF754
:100F20008DF904F0E3F80448C46904F00C0008B13A
:100F30000220EFE70020EDE700F00A40005800F043
:100F40002DE9F04107460E46144600BF2C4885693E
:100F500005F001000028F9D1B00929494860C6F31D
:100F600083008860A40838E02648006826490840C5
:100F70002649884206D12348006880B210B930461D
:100F800004F094F81E49386848610A20FFF756F9C2
:100F900000BF1B48856905F001000028F9D105F064
:100FA000100078B11748006817490840174988426F
:100FB00005D11448006880B208B904F05BF82846EF
:100FC000BDE8F0813F1D641E3CB10D48806820B92A
:100FD0000B484068401C0A494860002CC4D10948AD
:100FE0000068094908400949884205D10548006858
:100FF00080B208B904F03EF801488069E0E70000DB
:1010000000F00A4000E00F400000FF7000000510F3
:1010100010B58B090B4C6360C1F38303A360920886
:101020000DE0084B5B690360001D521E3AB1054B91
:101030009B6823B9034B5B685B1C024C6360002A0E
:10104000EFD110BD00F00A4010B50346CC00443487
:1010500018591070040A5470040C9470040ED47063
:10106000CC00403418591071040A547110BD10B5E9
:10107000CB004033C3586FF30F03147923435479E3
:1010800043EA0424CB004033C4501378547843EA35
:101090000423947843EA0443D47843EA0464CB00FD
:1010A0004433C45010BD000070B5D0F8185C156012
:1010B00005680C4E35400D60D0F8DC4004F48035F6
:1010C0001DB1C4F30D051D600AE0056805F4801527
:1010D0001DB14FF420551D6002E04FF400651D6006
:1010E00070BD0000FF7E5F7A30B504680A4D2C4069
:1010F0000C4344F40044046023B143F48034C0F84A
:10110000DC4005E0D0F8DC4024F48034C0F8DC405A
:10111000C0F8182C30BD00000C81A0854268024B3D
:101120001A400A434260704700F8FE7FF0B504465B
:10113000DDE9055700BFDFF894C0DCF800C00CF013
:10114000010CBCF1000FF6D142EA870C4CF0800094
:10115000202D01D8202B03D940F08070ED08DB084A
:10116000AB4202D140EA052007E04FF4000C4CEA04
:10117000052C4CEA434C4CEA0000C4F8000CDFF8A4
:1011800050C0DCF8146000200DE0DFF844C05CF8CB
:1011900030C08C4506D3DFF838C00CEBC00CDCF84F
:1011A000046002E0401C0328EFD300BFD4F810C055
:1011B0002CF03C0C4CEA060CC4F810C04FF0FF3C7D
:1011C000C4F80CC1C4F810C1F0BD000000CC0E4042
:1011D000B8B0000044F245020A400AB141F480313F
:1011E00042F2BA720A400AB141F4004121F00042D1
:1011F0001AB121F00042C0F8142C01F000422AB1CB
:10120000D0F8D82F42F00102C0F8D82F704744F22E
:1012100045020A400AB141F4803142F2BA720A40F2
:101220000AB141F4004121F0004232B1D0F81C2C47
:1012300021F000431A43C0F81C2C01F000422AB1EF
:10124000D0F8D42F42F00102C0F8D42F704700002C
:1012500010B50246D2F8140C094C204021B1D2F846
:101260001C4C44F0F044204011B1D2F8D83F01E0CA
:10127000D2F8D03F03F001040CB140F0004010BDA3
:10128000FFFF01FC70B505460C46C5F8C44F04F0DD
:10129000404060B9134803F0BBFD00BF114803F0A4
:1012A0009BFD0028FAD042F21070FEF7C7FF04F051
:1012B0004040B0F1404F06D10B48006840F4803008
:1012C0000949086005E00848006820F480300649B4
:1012D0000860064800F042F84FF47A70FEF7AEFF5F
:1012E00070BD0000003000F0C8CF0E4000C00E40BE
:1012F000034600BF186900F001000028FAD1186900
:1013000000F03C0040EA821040EAC120401C186115
:1013100000BF186900F001000028FAD1586980B2B6
:10132000704710B500BF046904F00104002CFAD125
:101330004361046904F03C0444EA821444EAC12491
:10134000E41C046100BF046904F00104002CFAD11C
:1013500010BD0146C86A00F061007047D0F8001C5B
:1013600041F00101C0F8001C00BFD0F8001C01F0E2
:1013700001010029F9D17047C0F80C1C7047D0F862
:10138000181C41F00201C0F8181C016841F004016A
:10139000016070470146D1F828077047C0F8101C5B
:1013A00070470021C0F8041C7047D0F8181C41F4A5
:1013B0000051C0F8181C016841F008010160704735
:1013C00002F001031BB1D0F800340B4302E0D0F867
:1013D00000348B43C0F8003402F002031BB1D0F894
:1013E00020340B4302E0D0F820348B43C0F8203483
:1013F00070470000F0B55F4D2D685F4E35405F4E81
:10140000B5421AD0002416E00125A5400D4085B153
:10141000D0F8C45F67000326BE40B543C0F8C45F80
:10142000D0F8C45F6700C2F34116BE403543C0F830
:10143000C45F651CECB2082CE6DB02F001051DB1AF
:10144000D0F800550D4302E0D0F800558D43C0F8A8
:10145000005502F002051DB1D0F804550D4302E01D
:10146000D0F804558D43C0F8045502F004051DB1B1
:10147000D0F808550D4302E0D0F808558D43C0F868
:10148000085502F008051DB1D0F818550D4302E0CB
:10149000D0F818558D43C0F81855364D2D68364E86
:1014A0003540364EB5420BD002F010051DB1D0F8D4
:1014B0003C550D4302E0D0F83C558D43C0F83C55F7
:1014C00003F001051DB1D0F80C550D4302E0D0F832
:1014D0000C558D43C0F80C5503F002051DB1D0F832
:1014E00010550D4302E0D0F810558D43C0F810554B
:1014F00003F004051DB1D0F814550D4302E0D0F8F7
:1015000014558D43C0F8145503F008051DB1D0F8EB
:101510001C550D4302E0D0F81C558D43C0F81C55F6
:10152000144D2D68144E3540144EB54217D003F4B7
:1015300000751DB1D0F844550D4302E0D0F8445574
:101540008D43C0F8445503F440751DB1D0F84055A3
:101550000D4302E0D0F840558D43C0F840551BB90B
:10156000D0F828550D4302E0D0F828558D43C0F837
:101570002855F0BD00E00F400000FF70000005108E
:1015800010B50146C1F307400F4BDB6E01248440C8
:10159000234033B1012303EB40030C4C54F82300E8
:1015A00003E04300094C54F82300C1F30722D0F8AC
:1015B0002C350F249440A34301F00F04944023439F
:1015C000C0F82C3510BD000000E00F4068B20000EC
:1015D00030B504460D46022229462046FFF7F0FEAC
:1015E0000823662229462046FFF704FF30BD30B5A8
:1015F00004460D46022229462046FFF7E1FE092354
:10160000012229462046FFF7F5FE30BD30B50446DD
:101610000D46022229462046FFF7D2FE082301226A
:1016200029462046FFF7E6FE30BD002303EB810389
:10163000C25070470146486800F0010008B101201F
:1016400070470020FCE7416070470146886870479A
:1016500081607047016A41F01001016270470246E3
:10166000516801F0010008B10020704701F012003C
:1016700010B101F01C00F8E70020F6E770B5034652
:101680000C4616461846FFF7E5FF012E01D10F4A1A
:1016900000E00F4A142000FB0240401E02EB8201D2
:1016A0008900B0FBF1F0451EDD60D3F8C00F00F0FB
:1016B000010048B107482044401E0649B0FBF1F044
:1016C000451E45F08000D86070BD0000801A0600FD
:1016D000A08601008047370142EA4103036070475A
:1016E000016A41F0200101620121C0F8041870472D
:1016F00000B502460B461046FFF7F2FFC2F800386D
:1017000000BD10B5044614B94FF0FF3010BDA069FC
:1017100008B1E06910B94FF0FF30F7E7902120469B
:1017200000F01CF80021204600F002F80020EDE750
:10173000F8B504460D4608208DF800008DF80150DC
:10174000A07D02236A466F21E769B84746B2002EA2
:1017500002DA4FF0FF30F8BD0020FCE7F8B5044690
:101760000D4607208DF800008DF80150A07D022362
:101770006A466F21E769B84746B2002E02DA4FF099
:10178000FF30F8BD0020FCE710B5002426E0002063
:1017900004EBC4014A4A02EB8101086204EBC40174
:1017A00002EB8101486004EBC40102EB8101886017
:1017B000172C01D1104605E0601C00EBC000404929
:1017C00001EB800004EBC4013D4A02EB8101C860DB
:1017D0003C4804EBC40142F82100641C182CD6D309
:1017E000002039498860C860002459E0032240F293
:1017F000EC51104605F02AFB04EBC401334A02EB1E
:10180000810108624FF4804004EBC40102EB8101C6
:10181000486004EBC400114601EB8000006A18B375
:1018200004EBC40001EB8000006A406804EBC401D3
:1018300002EB8101886004EBC400114601EB8000DB
:10184000406804EBC40102EB8101096A498908433D
:1018500004EBC40102EB810148604FF0004004EB4F
:10186000C40142F821000AE0002004EBC401174A39
:1018700002EB8101886004EBC40142F82100072CCF
:1018800001D1124805E0601C00EBC0000F4901EBDC
:10189000800004EBC4010D4A02EB8101C860641CA6
:1018A000082CA3D3002008498860C860074908486D
:1018B000FFF762FD02490648FFF770FD10BD00000A
:1018C000B82A01200000D04020010020182E01205D
:1018D00000C00E40042806D11949096841F480313E
:1018E000174A11602BE0052806D11549096841F413
:1018F0000031134A116022E0062806D11049096818
:1019000041F480210E4A116019E00F2808D14FF0F0
:10191000E021096941F002014FF0E02211610EE07F
:1019200010280CD3A0F1100101F01F0201219140F9
:10193000A0F110025209034B53F8222011607047A6
:1019400024ED00E0B4B3000010B5FEF763FC08B16D
:10195000012010BD0020FCE710B5FEF762FC08B1C5
:10196000012010BD0020FCE710B5084803F0FEF987
:1019700000BF064803F030FA0028FAD0FFF7BEFA9D
:1019800004460CB100BFFEE710BD0000005800F097
:101990002DE9F04104460D46164604F0030018B147
:1019A0004FF0FF30BDE8F0810027FEF78BFC0746C3
:1019B000324621462846FFF72BFB3846FEF786FCC9
:1019C0000020EFE72DE9F04104460D46164604F0ED
:1019D000030018B14FF0FF30BDE8F0810027FEF79B
:1019E00071FC0746324621462846FFF7A9FA20B186
:1019F000324621462846FFF7A3FA3846FEF766FC32
:101A00000020E9E72DE9F04104460D4616461F4641
:101A1000082C03DB4FF0FF30BDE8F08100BF04EB82
:101A20004400EC4901EB8000C0780128F7D004EBBA
:101A3000440001EB800000790128F0D0002004EB85
:101A40004401E44A02F8210004EB4400114601EB92
:101A50008000467004EB440001EB8000877004EBCB
:101A6000440001EB8000856014BBDB4803F07EF985
:101A7000DA4803F07BF9D94803F078F9D848FFF742
:101A80007FFDD848FFF77CFD0421D748FFF7BEFD56
:101A90000821D548FFF7ABFDA6B9D448854208D147
:101AA00003F0F8F9804600224146D148FFF7E6FDF1
:101AB0000CE003F0EFF9804601224146CC48FFF7E5
:101AC000DDFD03E03946CA48FFF712FE012C33D191
:101AD000C148401C03F04AF9C048401D03F046F9D4
:101AE000BE48401D03F042F9C248FFF749FDC24815
:101AF000FFF746FD0121C148FFF788FD0221BF48DD
:101B0000FFF775FDA6B9B948854208D103F0C2F9BF
:101B1000804600224146BA48FFF7B0FD0CE003F0D2
:101B2000B9F9804601224146B548FFF7A7FD03E019
:101B30003946B348FFF7DCFD022C33D1A648801CA0
:101B400003F014F9A548093003F010F9A34809304F
:101B500003F00CF9AB48FFF713FDAB48FFF710FD9E
:101B60000221AA48FFF752FD0121A848FFF73FFDD7
:101B7000A6B99E48854208D103F08CF98046002220
:101B80004146A348FFF77AFD0CE003F083F9804655
:101B9000012241469E48FFF771FD03E039469C480B
:101BA000FFF7A6FD032C33D18B48C01C03F0DEF8F1
:101BB0008A48083003F0DAF88848083003F0D6F88D
:101BC0009448FFF7DDFC9448FFF7DAFC10219348B6
:101BD000FFF71CFD20219148FFF709FDA6B98348B6
:101BE000854208D103F056F98046002241468C48D0
:101BF000FFF744FD0CE003F04DF980460122414619
:101C00008748FFF73BFD03E039468548FFF770FD45
:101C1000042C33D17048001D03F0A8F86F48083039
:101C200003F0A4F86D48083003F0A0F87D48FFF7F2
:101C3000A7FC7D48FFF7A4FC40217848FFF7E6FCAD
:101C400080217648FFF7D3FCA6B96848854208D1C1
:101C500003F020F98046002241467448FFF70EFD4C
:101C60000CE003F017F98046012241466F48FFF768
:101C700005FD03E039466D48FFF73AFD052C31D1EB
:101C80005548401D03F072F8544803F06FF853486C
:101C900003F06CF86648FFF773FC6648FFF770FCCA
:101CA00001215148FFF7B2FC02214F48FFF79FFC8A
:101CB000A6B94E48854208D103F0ECF880460022D0
:101CC00041465D48FFF7DAFC0CE003F0E3F880469C
:101CD000012241465848FFF7D1FC03E039465648F7
:101CE000FFF706FD062C37D13B48801D03F03EF878
:101CF0003A48401E03F03AF83848401E03F036F8E0
:101D000041F60200FFF73CFC41F60240FFF738FCC9
:101D100040214FF04020FFF779FC80214FF0402018
:101D2000FFF765FCA6B93148854208D103F0B2F847
:101D30008046002241464148FFF7A0FC0CE003F03A
:101D4000A9F88046012241463C48FFF797FC03E092
:101D500039463A48FFF7CCFC072C33D11E48C01D4A
:101D600003F004F81D48801C03F000F81B48801C99
:101D700002F0FCFF3248FFF703FC3248FFF700FC9B
:101D800001213148FFF742FC02212F48FFF72FFCC9
:101D9000A6B91648854208D103F07CF88046002297
:101DA00041462A48FFF76AFC0CE003F073F88046CE
:101DB000012241462548FFF761FC03E039462348EC
:101DC000FFF796FC012004EB4401024A02F82100CF
:101DD000002021E6AC2D0020002000F0010800F0DA
:101DE00002080100020C010000500040A086010022
:101DF00000000240020006000204060000600240EB
:101E00000010024002040A0002000A0000200640FE
:101E100000200240021009000214090000100640D0
:101E20000030024002180900021C090000000C40AA
:101E3000020001000204010000100C4000200C40D0
:101E400002000300020403000070004000300C4058
:101E50002DE9F0470546884617461E464FF0000913
:101E6000082D03DB4FF0FF30BDE8F08737B12EB10E
:101E700005EB4500FA4911F8200010B94FF0FF308A
:101E8000F2E7FEF71FFA8146012005EB4501F44A0F
:101E900002EB8101C87005EB4500114601EB8000A3
:101EA0004078002878D1002D78D100BFED48FFF7A9
:101EB000C1FB0028FAD101224146EA48FFF70CFC99
:101EC000012E29D10721E748FFF7BDFBE548FFF7C1
:101ED000C6FB58B1002005EB4501E14A02EB810148
:101EE000C8704846FEF7F2F9B01EBDE700BFDD48F6
:101EF000FFF7A0FB0028FAD1DA48FFF7A6FB3870FD
:101F0000002005EB4501D64A02EB8101C870484626
:101F1000FEF7DCF90020A7E700243BE024B90B2101
:101F2000D048FFF790FB0BE0701EA04204D10521C2
:101F3000CC48FFF788FB03E00921CA48FFF783FB81
:101F4000C848FFF78CFBD0B1701EA0420AD0C5482C
:101F5000FFF785FB00F01000102803D00421C148D2
:101F6000FFF771FB002005EB4501BD4A02EB810143
:101F7000C8704846FEF7AAF94FF0FF3074E700BF7B
:101F8000B848FFF757FB0028FAD1B648FFF75DFBCA
:101F90003855641CB442C1D365E3FFE7012D78D105
:101FA00000BFB148FFF746FB0028FAD101224146A5
:101FB000AD48FFF791FB012E29D10721AA48FFF771
:101FC00042FBA948FFF74BFB58B1002005EB450148
:101FD000A34A02EB8101C8704846FEF777F9B01EAC
:101FE00042E700BFA048FFF725FB0028FAD19E4832
:101FF000FFF72BFB3870002005EB4501984A02EBF8
:102000008101C8704846FEF761F900202CE70024E2
:102010003BE024B90B219448FFF715FB0BE0701E41
:10202000A04204D105219048FFF70DFB03E00921F0
:102030008D48FFF708FB8C48FFF711FBD0B1701EED
:10204000A0420AD08848FFF70AFB00F010001028D1
:1020500003D004218448FFF7F6FA002005EB450180
:102060007F4A02EB8101C8704846FEF72FF94FF016
:10207000FF30F9E600BF7C48FFF7DCFA0028FAD110
:102080007948FFF7E2FA3855641CB442C1D3EAE25A
:10209000FFE7022D78D100BF7448FFF7CBFA002884
:1020A000FAD1012241467148FFF716FB012E29D1D2
:1020B00007216E48FFF7C7FA6C48FFF7D0FA58B10E
:1020C000002005EB4501664A02EB8101C8704846D5
:1020D000FEF7FCF8B01EC7E600BF6448FFF7AAFA97
:1020E0000028FAD16148FFF7B0FA3870002005EBFC
:1020F00045015B4A02EB8101C8704846FEF7E6F8ED
:102100000020B1E600243BE024B90B215748FFF73B
:102110009AFA0BE0701EA04204D105215348FFF744
:1021200092FA03E009215148FFF78DFA4F48FFF773
:1021300096FAD0B1701EA0420AD04C48FFF78FFA31
:1021400000F01000102803D004214848FFF77BFA64
:10215000002005EB4501424A02EB8101C870484668
:10216000FEF7B4F84FF0FF307EE600BF3F48FFF7C0
:1021700061FA0028FAD13D48FFF767FA3855641C28
:10218000B442C1D36FE2FFE7032D73D100BF3848DB
:10219000FFF750FA0028FAD1012241463448FFF7F0
:1021A0009BFA012E29D107213148FFF74CFA30481C
:1021B000FFF755FA58B1002005EB4501284A02EB1C
:1021C0008101C8704846FEF781F8B01E4CE600BF9A
:1021D0002748FFF72FFA0028FAD12548FFF735FAEC
:1021E0003870002005EB45011D4A02EB8101C870E3
:1021F0004846FEF76BF8002036E6002446E024B996
:102200000B211B48FFF71FFA0BE0701EA04204D100
:1022100005211748FFF717FA03E009211448FFF7D3
:1022200012FA1348FFF71BFA28B3701EA0420AD017
:102230000F48FFF714FA00F01000102803D0042113
:102240000B48FFF700FA002005EB4501044A02EBBA
:102250008101C8704846FEF739F84FF0FF3003E6B9
:10226000AC2D00200000024000100240002002407F
:10227000003002400DE000BFFE48FFF7DBF9002808
:10228000FAD1FC48FFF7E1F93855641CB442B6D3E3
:10229000E9E1042D78D100BFF748FFF7CBF900281A
:1022A000FAD101224146F448FFF716FA012E29D14E
:1022B0000721F148FFF7C7F9EF48FFF7D0F958B108
:1022C000002005EB4501ED4A02EB8101C87048464C
:1022D000FDF7FCFFB01EC7E500BFE748FFF7AAF90E
:1022E0000028FAD1E448FFF7B0F93870002005EB78
:1022F0004501E24A02EB8101C8704846FDF7E6FF5E
:102300000020B1E500243BE024B90B21DA48FFF7B7
:102310009AF90BE0701EA04204D10521D648FFF7C0
:1023200092F903E00921D448FFF78DF9D248FFF76D
:1023300096F9D0B1701EA0420AD0CF48FFF78FF9AE
:1023400000F01000102803D00421CB48FFF77BF9E0
:10235000002005EB4501C94A02EB8101C8704846DF
:10236000FDF7B4FF4FF0FF307EE500BFC248FFF736
:1023700061F90028FAD1C048FFF767F93855641CA5
:10238000B442C1D36FE1FFE7052D78D100BFBC484F
:10239000FFF750F90028FAD101224146B848FFF76B
:1023A0009BF9012E29D10721B548FFF74CF9B44814
:1023B000FFF755F958B1002005EB4501AF4A02EB94
:1023C0008101C8704846FDF781FFB01E4CE500BF93
:1023D000AB48FFF72FF90028FAD1A948FFF735F9E4
:1023E0003870002005EB4501A44A02EB8101C8705A
:1023F0004846FDF76BFF002036E500243BE024B99A
:102400000B219F48FFF71FF90BE0701EA04204D17B
:1024100005219B48FFF717F903E009219848FFF7CA
:1024200012F99748FFF71BF9D0B1701EA0420AD0ED
:102430009348FFF714F900F01000102803D004218E
:102440008F48FFF700F9002005EB45018B4A02EBAE
:102450008101C8704846FDF739FF4FF0FF3003E5B2
:1024600000BF8748FFF7E6F80028FAD18448FFF755
:10247000ECF83855641CB442C1D3F4E0FFE7062DF4
:1024800078D100BF7F48FFF7D5F80028FAD10122A4
:1024900041467C48FFF720F9012E29D107217948D0
:1024A000FFF7D1F87748FFF7DAF858B1002005EBCD
:1024B0004501724A02EB8101C8704846FDF706FFEC
:1024C000B01ED1E400BF6F48FFF7B4F80028FAD17E
:1024D0006C48FFF7BAF83870002005EB4501674AF1
:1024E00002EB8101C8704846FDF7F0FE0020BBE416
:1024F00000243BE024B90B216248FFF7A4F80BE06D
:10250000701EA04204D105215E48FFF79CF803E04D
:1025100009215C48FFF797F85A48FFF7A0F8D0B1B7
:10252000701EA0420AD05748FFF799F800F010003B
:10253000102803D004215348FFF785F8002005EB4D
:1025400045014E4A02EB8101C8704846FDF7BEFEC8
:102550004FF0FF3088E400BF4A48FFF76BF80028CF
:10256000FAD14848FFF771F83855641CB442C1D31A
:1025700079E0FFE7072D76D100BF4348FFF75AF80F
:102580000028FAD1012241463F48FFF7A5F8012E65
:1025900029D107213C48FFF756F83B48FFF75FF881
:1025A00058B1002005EB4501344A02EB8101C870A7
:1025B0004846FDF78BFEB01E56E400BF3248FFF7D9
:1025C00039F80028FAD13048FFF73FF8387000207A
:1025D00005EB4501294A02EB8101C8704846FDF729
:1025E00075FE002040E400243BE024B90B2126487E
:1025F000FFF729F80BE0701EA04204D10521224804
:10260000FFF721F803E009211F48FFF71CF81E48D7
:10261000FFF725F8D0B1701EA0420AD01A48FFF784
:102620001EF800F01000102803D004211648FFF710
:102630000AF8002005EB4501104A02EB8101C87041
:102640004846FDF743FE4FF0FF300DE400BF0E4853
:10265000FEF7F0FF0028FAD10B48FEF7F6FF3855D9
:10266000641CB442C1D3002005EB4501034A02EBD0
:1026700081010BE00030024000000C40AC2D002036
:1026800000100C4000200C4000300C40C870484640
:10269000FDF71CFE002028E42DE9F047054688469A
:1026A00016461F464FF00009082D03DB4FF0FF30A0
:1026B000BDE8F08736B12FB105EB4500F74911F8B9
:1026C000200010B94FF0FF30F2E7FDF7FBFD814627
:1026D000012005EB4501F14A02EB8101087105EB90
:1026E0004500114601EB80004078002876D1002D8E
:1026F00075D100BFEA48FEF79DFF0028FAD10022FD
:102700004146E748FEF7E8FF012F28D13178E44839
:10271000FEF79EFF0721E248FEF795FFE048FEF72F
:102720009EFF58B1002005EB4501DC4A02EB810118
:1027300008714846FDF7CAFDB81EB9E700BFD84882
:10274000FEF778FF0028FAD105EB4501D34A02EBEA
:10275000810108714846FDF7B9FD0020A8E7002473
:1027600045E044B9315DCE48FEF772FF0321CC4805
:10277000FEF769FF13E0781EA04208D1315DC8481A
:10278000FEF766FF0521C648FEF75DFF07E0315DF5
:10279000C348FEF75DFF0121C148FEF754FFC04862
:1027A000FEF75DFFE0B1781EA0420AD0BC48FEF7FC
:1027B00056FF00F01000102803D00421B848FEF79F
:1027C00042FF002005EB4501B44A02EB810108718C
:1027D0004846FDF77BFD4FF0FF3069E71CE209E05A
:1027E00000BFAF48FEF726FF0028FAD1641CBC42A8
:1027F000B7D3A5E3012D7FD100BFAA48FEF71AFF8A
:102800000028FAD100224146A648FEF765FF012FB5
:1028100028D13178A348FEF71BFF0721A148FEF716
:1028200012FFA048FEF71BFF58B1002005EB450141
:102830009A4A02EB810108714846FDF747FDB81E30
:1028400036E700BF9748FEF7F5FE0028FAD105EB02
:102850004501924A02EB810108714846FDF736FDB9
:10286000002025E7002444E044B9315D8D48FEF79F
:10287000EFFE03218B48FEF7E6FE13E0781EA04230
:1028800008D1315D8748FEF7E3FE05218548FEF754
:10289000DAFE07E0315D8348FEF7DAFE0121814868
:1028A000FEF7D1FE7F48FEF7DAFED8B1781EA042CF
:1028B0000AD07C48FEF7D3FE00F01000102803D0A9
:1028C00004217848FEF7BFFE002005EB4501734A5E
:1028D00002EB810108714846FDF7F8FC4FF0FF302C
:1028E000E6E609E000BF6F48FEF7A4FE0028FAD133
:1028F000641CBC42B8D323E3022D7FD100BF6A48D9
:10290000FEF798FE0028FAD1002241466648FEF7FD
:10291000E3FE012F28D131786348FEF799FE0721A5
:102920006148FEF790FE6048FEF799FE58B100201E
:1029300005EB4501594A02EB810108714846FDF754
:10294000C5FCB81EB4E600BF5748FEF773FE00286A
:10295000FAD105EB4501514A02EB81010871484665
:10296000FDF7B4FC0020A3E6002444E044B9315D47
:102970004D48FEF76DFE03214B48FEF764FE13E061
:10298000781EA04208D1315D4748FEF761FE05215F
:102990004548FEF758FE07E0315D4348FEF758FE14
:1029A00001214148FEF74FFE3F48FEF758FED8B1DF
:1029B000781EA0420AD03C48FEF751FE00F01000FD
:1029C000102803D004213848FEF73DFE002005EB17
:1029D0004501324A02EB810108714846FDF776FC59
:1029E0004FF0FF3064E609E000BF2F48FEF722FEFB
:1029F0000028FAD1641CBC42B8D3A1E2032D7CD1DB
:102A000000BF2A48FEF716FE0028FAD100224146F0
:102A10002648FEF761FE012F28D131782348FEF7C2
:102A200017FE07212148FEF70EFE2048FEF717FE8D
:102A300058B1002005EB4501184A02EB81010871ED
:102A40004846FDF743FCB81E32E600BF1748FEF7C4
:102A5000F1FD0028FAD105EB4501104A02EB810196
:102A600008714846FDF732FC002021E600244FE0C3
:102A700044B9315D0D48FEF7EBFD03210B48FEF72D
:102A8000E2FD1DE0781EA04212D1315D0748FEF73D
:102A9000DFFD05210548FEF7D6FD11E0AC2D002035
:102AA00000000240001002400020024000300240BE
:102AB000315DF848FEF7CCFD0121F648FEF7C3FD75
:102AC000F448FEF7CCFDE0B1781EA0420AD0F148F0
:102AD000FEF7C5FD00F01000102803D00421ED48DA
:102AE000FEF7B1FD002005EB4501EB4A02EB810149
:102AF00008714846FDF7EAFB00E00CE04FF0FF30BC
:102B0000D6E500BFE348FEF795FD0028FAD1641C26
:102B1000BC42ADD314E2042D7FD100BFDF48FEF7E5
:102B200089FD0028FAD100224146DC48FEF7D4FD99
:102B3000012F28D13178D948FEF78AFD0721D748DF
:102B4000FEF781FDD548FEF78AFD58B1002005EB60
:102B50004501D14A02EB810108714846FDF7B6FBF9
:102B6000B81EA5E500BFCD48FEF764FD0028FAD1E8
:102B700005EB4501C84A02EB810108714846FDF7A3
:102B8000A5FB002094E5002444E044B9315DC3482E
:102B9000FEF75EFD0321C148FEF755FD13E0781EE8
:102BA000A04208D1315DBD48FEF752FD0521BB486A
:102BB000FEF749FD07E0315DB848FEF749FD012108
:102BC000B648FEF740FDB548FEF749FDD8B1781E7E
:102BD000A0420AD0B148FEF742FD00F010001028D4
:102BE00003D00421AD48FEF72EFD002005EB450182
:102BF000A94A02EB810108714846FDF767FB4FF0D7
:102C0000FF3055E509E000BFA448FEF713FD00289A
:102C1000FAD1641CBC42B8D392E1052D7FD100BF2C
:102C20009F48FEF707FD0028FAD1002241469C4844
:102C3000FEF752FD012F28D131789948FEF708FDA3
:102C400007219748FEF7FFFC9548FEF708FD58B1AD
:102C5000002005EB4501904A02EB810108714846CE
:102C6000FDF734FBB81E23E500BF8D48FEF7E2FCFC
:102C70000028FAD105EB4501874A02EB8101087172
:102C80004846FDF723FB002012E5002444E044B948
:102C9000315D8348FEF7DCFC03218148FEF7D3FC5D
:102CA00013E0781EA04208D1315D7D48FEF7D0FCCC
:102CB00005217B48FEF7C7FC07E0315D7848FEF749
:102CC000C7FC01217648FEF7BEFC7548FEF7C7FC3D
:102CD000D8B1781EA0420AD07148FEF7C0FC00F0BF
:102CE0001000102803D004216D48FEF7ACFC002032
:102CF00005EB4501684A02EB810108714846FDF782
:102D0000E5FA4FF0FF30D3E409E000BF6448FEF776
:102D100091FC0028FAD1641CBC42B8D310E1062D06
:102D20007FD100BF5F48FEF785FC0028FAD1002262
:102D300041465C48FEF7D0FC012F28D13178594834
:102D4000FEF786FC07215748FEF77DFC5548FEF745
:102D500086FC58B1002005EB45014F4A02EB81018A
:102D600008714846FDF7B2FAB81EA1E400BF4D480D
:102D7000FEF760FC0028FAD105EB4501464A02EB5C
:102D8000810108714846FDF7A1FA002090E4002473
:102D900044E044B9315D4348FEF75AFC0321414801
:102DA000FEF751FC13E0781EA04208D1315D3D488A
:102DB000FEF74EFC05213B48FEF745FC07E0315D80
:102DC0003848FEF745FC01213648FEF73CFC354803
:102DD000FEF745FCD8B1781EA0420AD03148FEF774
:102DE0003EFC00F01000102803D004212D48FEF70F
:102DF0002AFC002005EB4501274A02EB81010871FE
:102E00004846FDF763FA4FF0FF3051E409E000BF98
:102E10002448FEF70FFC0028FAD1641CBC42B8D34A
:102E20008EE0072D7DD100BF1F48FEF703FC002870
:102E3000FAD1002241461C48FEF74EFC012F35D145
:102E400031781948FEF704FC07211748FEF7FBFB11
:102E50001548FEF704FC58B1002005EB45010E4A69
:102E600002EB810108714846FDF730FAB81E1FE4F5
:102E700000BF0D48FEF7DEFB0028FAD105EB450147
:102E8000054A02EB810108714846FDF71FFA002050
:102E90000EE4000000300240AC2D002000000C4089
:102EA00000100C4000200C4000300C40002445E095
:102EB00044B9315D2848FEF7CBFB03212648FEF7D5
:102EC000C2FB13E0781EA04208D1315D2248FEF714
:102ED000BFFB05212048FEF7B6FB07E0315D1E4829
:102EE000FEF7B6FB01211C48FEF7ADFB1A48FEF7C2
:102EF000B6FBE0B1781EA0420AD01748FEF7AFFB40
:102F000000F01000102803D004211348FEF79BFBAB
:102F1000002005EB4501114A02EB8101087148468A
:102F200000E00DE0FDF7D2F94FF0FF3005E400BFFF
:102F30000948FEF77FFB0028FAD1641CBC42B7D3D6
:102F4000002005EB4501054A02EB81010871484666
:102F5000FDF7BCF9002040E400300C40AC2D00200F
:102F60007047000010B504462CB9012211460548EF
:102F7000FEF75BFB04E0FE2201210248FEF755FB51
:102F800010BD00000070004010B504462CB90222AC
:102F900011460548FEF749FB04E0FD2202210248E4
:102FA000FEF743FB10BD00000070004010B50E4856
:102FB00001F0DCFE012211460C48FEF701FA08235D
:102FC000012211460948FEF715FA074801F0CEFE26
:102FD000012202210548FEF7F3F90823012202210C
:102FE0000248FEF707FA10BD030800F00070004029
:102FF00010B5FFF7B5FFFFF7D9FFFEF7ADFCFEF701
:10300000B3FC10BD30B505460C46224600212846CB
:1030100000F026F830BD00000D480E490160014661
:10302000416000218160C160016141618161C161D4
:1030300001620163C162416207498163C1634FF468
:103040008061016441640146044A116070470000D8
:103050009427002048454150DC2700206C000020C8
:103060002DE9F04103460C4617460FB9BDE8F08143
:1030700003B9FBE70025002202E02D022543521C84
:10308000042AFAD3384603F0030C1946BCF1000FAA
:1030900008D0624603E001F8014B401E521C08B103
:1030A000042AF8D30E4601E020C6001F0428FBD2F4
:1030B000314602E001F8014B401E0028FAD100BF62
:1030C000D4E700001D481E481E481F481F482048DE
:1030D00020482148214822482248234823482448A0
:1030E0002448254825482648264827482748284870
:1030F0002848294829482A482A482B482B482C4840
:103100002C482D482D482E482E482F482F4830480F
:1031100030483148314832483248334833483448DF
:1031200034483548354836483648374837483848AF
:1031300038483948394800BF7047000004B40000DF
:1031400008B400000EB4000010B400000CB400007D
:1031500012B4000014B4000016B4000018B400004B
:103160001AB400001CB400001EB4000020B400001B
:1031700022B4000024B4000026B4000028B40000EB
:103180002AB400002CB400002EB4000030B40000BB
:1031900032B4000034B4000036B4000038B400008B
:1031A0003AB400003CB400003EB4000040B400005B
:1031B00042B4000044B4000046B4000048B400002B
:1031C0004AB400004CB400004EB4000050B40000FB
:1031D00052B4000054B4000056B400005AB40000C9
:1031E0005CB400005EB4000060B40000D422002093
:1031F0005427002064B4000066B4000068B40000E6
:103200006AB400006CB400006EB4000070B400003A
:1032100072B4000074B4000062B4000076B4000020
:103220002DE9F04105460E46144600271148007866
:1032300018B112202070BDE8F0812878012808D04C
:10324000022807D0032802D0042804D100E000BFE0
:1032500000BF00BF02E001202070ECE700BFFDF7D7
:1032600031F807466E613846FDF730F800202070CF
:1032700000BFE0E72100002010B500F019F801F0D0
:1032800051FA01F07DFA01F09DFA01F01BFA01F00C
:10329000DBF901F031FB01F05BFB01F0D3FA01F047
:1032A000F9FA00F0A1FF00F01FF8FFF70BFF10BDC7
:1032B0000948802102E0491E002204C00029FAD1F9
:1032C000064A074B1A601A46126822F007021A6073
:1032D0000022044B1A8070478C0100208C030020D0
:1032E00000000020040000207047000010B50024FA
:1032F000FCF7E8FF044608480078012808D1074891
:103300000078FF2804D205480078401C0349087063
:103310002046FCF7DBFF10BD2E000020210000201E
:1033200010B500241A480078012830D1FCF7CAFFF4
:1033300004461848007820B116480078401E154908
:10334000087014480078F8B913480078E0B901F023
:1033500061FB12481249097850F8210011490860B0
:103360000F4800781049097888420DD00D48006850
:10337000C06B401C0B490968C8630C480068401CBE
:103380000A490860FCF7BEFF2046FCF79FFF10BD0E
:103390002E0000202100002022000020140E00201A
:1033A000240000203C000020230000200800002012
:1033B0002DE9FC5F05460F4691469A460020009095
:1033C000FCF780FF009018480468006820B1164898
:1033D00000684068144908600098FCF777FF2CB932
:1033E0005A208AF800000020BDE8FC9FA8462E461F
:1033F000781E01904FF0000B05E04E44C8F80060C5
:10340000B0460BF1010B01988345F6D30020C8F8B4
:103410000000256065602761E760C4F808908AF8BD
:1034200000002046E0E70000480000202DE9F041C0
:1034300004460D460027FCF745FF0746206968B1A2
:103440006668306860602069401E20613846FCF77D
:103450003DFF002028703046BDE8F0813846FCF77B
:1034600035FF5D2028700020F6E770B504460D4654
:103470000026FCF727FF0646D4E90310884204D350
:103480003046FCF723FF5E2070BD606828606560F1
:103490002069401C20613046FCF718FF0020F3E74C
:1034A0002DE9F04106460F464FF00008204800780D
:1034B00010B10020BDE8F081FCF704FF80461D48F4
:1034C0000468006820B11B4800684068194908601A
:1034D0004046FCF7FBFEFCB1FCF7F4FE80461648C4
:1034E0000568D5B100680068134908604046FCF7DC
:1034F000EDFE6E6006EB8700A860EE602E61AF8285
:103500000020E882022020700020208165600BA04E
:103510006061204601F08AF808E0064800686060B3
:10352000044804604046FCF7D1FE00242046C1E771
:10353000210000200C0000204C0000203F00000073
:103540002DE9F0470746884615464FF000093878C0
:10355000022804D0012028700020BDE8F0873E48F2
:10356000007818B1022028700020F6E73B48007868
:1035700018B10D2028700020EFE7FCF7A3FE81466C
:103580007C68E08A98B12169081D20610E68E08A94
:10359000401EE082A1682069884201D160682061F4
:1035A0004846FCF793FE002028703046D5E72C48AB
:1035B000006890F8340040F004002949096881F857
:1035C000340000202649096881F835002448006845
:1035D000C0F83080384600F0EBFF4846FCF776FE36
:1035E00001F0DEF9FCF76EFE81461D48006890F898
:1035F000350020B101280DD002280AD105E0184875
:103600000068466A002028700DE000260E20287011
:1036100009E000BF39461248006800F095FF002617
:103620000A20287000BF00BF00200D49096881F8FA
:1036300034000B49096881F8350009490968C861F7
:103640000749096808620649096848624846FCF764
:103650003DFE304681E700002100002022000020CE
:10366000340000202DE9F04105460E460027287859
:10367000022802D00120BDE8F081FCF723FE0746B6
:10368000A87A60B1002304223146284600F014FFD6
:103690003846FCF71BFE01F083F90020EBE76C686D
:1036A000E08AA18A884204DB3846FCF70FFE1E2020
:1036B000E1E7E168081DE0600E60E08A401CE082FE
:1036C000D4E90210884201D16068E0603846FCF716
:1036D000FDFD0020CFE72DE9F04705460C464FF0F1
:1036E000000A2878022802D00120BDE8F087FCF704
:1036F000E9FD8246A87A207405F10B0804F1080957
:10370000002705E018F8010B09F8010B781CC7B277
:10371000082FF7D36E68F08A18B13069006820600E
:1037200001E000202060F08AA080B08AE08050464E
:10373000FCF7CCFD0020D8E710B500240B4800783A
:10374000012811D1FCF7BEFD04460948007840B9B4
:1037500008480078FF2804D206480078401C054934
:1037600008702046FCF7B2FD10BD00002E000020BE
:10377000210000202200002010B50024134800780A
:10378000012821D1FCF79EFD044611480078C0B9FC
:103790001048007888B10F480078401E0D49087025
:1037A0000846007828B92046FCF790FD01F0F8F8AB
:1037B0000AE02046FCF78AFD06E02046FCF786FD7D
:1037C00002E02046FCF782FD10BD00002E00002024
:1037D000210000202200002070B505460026104878
:1037E000007808B1002070BDFCF76CFD06460D485E
:1037F0000468006820B10B48006840680949086007
:103800003046FCF763FD4CB1032020702581002079
:10381000606005A06061204600F008FF2046E2E7F6
:10382000210000200C0000203F0000002DE9F041A5
:1038300005460E46144600272878032803D00120A9
:103840002070BDE8F0813248007810B1022020706D
:10385000F7E73048007810B10D202070F1E7FCF751
:1038600031FD0746288940B12889401E2881384605
:10387000FCF72CFD00202070E3E72748006890F853
:10388000340040F001002449096881F83400002028
:103890002149096881F835001F48006806632846F9
:1038A00000F086FE3846FCF711FD01F079F8FCF7D0
:1038B00009FD07461848006890F8350020B1012836
:1038C00009D0022806D102E0002020700BE00E2073
:1038D000207008E000BF29460F48006800F034FE61
:1038E0000A20207000BF00BF00200B49096881F842
:1038F00034000949096881F8350007490968C86139
:103900000549096808623846FCF7E0FC00BF98E703
:1039100021000020220000203400002070B5044661
:1039200000252078032801D0012070BDFCF7CAFCD7
:103930000546A07A60B1002301221946204600F016
:10394000BBFD2846FCF7C2FC01F02AF80020ECE79A
:1039500020894FF6FF71884207D22089401C2081C0
:103960002846FCF7B3FC0020DFE72846FCF7AEFC56
:103970003320DAE710B50B48007890B901F04AF827
:10398000094800780949087009480749097850F83A
:103990002100084908600846006807490860FCF7EC
:1039A00098FC10BD2E0000202400002023000020E1
:1039B000140E00203C0000203400002010B500242C
:1039C000022000F035FBFCF77DFC044600200B498B
:1039D00008602046FCF77AFC642000F029FBFCF725
:1039E00071FC044605480068054908600120054946
:1039F00008702046FCF76AFC10BD00003000002073
:103A0000180000202000002010B504462046FCF7D6
:103A100003FE10BD2DE9F04F85B081468A469346DE
:103A20001C46DDE90F78129D00200390FCF74AFC4C
:103A300003902348007830B10398FCF747FC3C2002
:103A400005B0BDE8F08F1F4850F8240088BB012066
:103A50001C4941F824000398FCF738FC2A464146EB
:103A6000384601F01BF92B465A465146484600F0AD
:103A700073F904901198CDE9008002953A462046EA
:103A80000E9B049900F0DCFF064636B90E4800781C
:103A900001280CD100F084FF09E0FCF713FC03902F
:103AA0000020084941F824000398FCF70FFC304639
:103AB000C6E7FFE70398FCF709FC2820C0E70000F1
:103AC00021000020140E00202E00002010B5044616
:103AD0002046FCF7A2FD10BD2DE9F0410546002768
:103AE0004A48007810B14020BDE8F0813F2D01D157
:103AF0003E20F9E7FCF7E6FB0746FF2D03D14448DB
:103B0000006890F83650434850F8254024B93846AC
:103B1000FCF7DCFB4320E7E7012C04D13846FCF737
:103B2000D5FB3D20E0E714F8380F3B49085C61788D
:103B300088432178384A505414F838091146085CF3
:103B400030B994F83A103548007888433349087002
:103B5000E06918B12046E16900F0F6FC206A18B16E
:103B60002046216A00F007FDA66A16B1304600F033
:103B700097FD0020206384F8340084F8350028483D
:103B80000078FF2804D226480078401C2449087099
:103B90003846FCF79BFB00F08DFCFCF793FB0746D7
:103BA0001F48007820B11E480078401E1C4908704C
:103BB000204600F041F81B480078401E1949087063
:103BC0000020144941F82500A06930B9002061693E
:103BD000886115496069086005E0D4E9050148611C
:103BE000D4E9051088611148006860610F480460DD
:103BF0000FA020653846FCF769FB0E4800780128C5
:103C000001D100F0CDFE00206EE700002100002071
:103C100034000020140E0020260000202500002083
:103C2000220000202F00002040000020380000204B
:103C30003F0000002E00002010B504462046FCF78F
:103C4000EDFC10BD10B5FCF7EAFC10BD2DE9F0410C
:103C500006460F4614464FF000081548007818B184
:103C600012202070BDE8F081FCF72CFB8046FF2E6F
:103C700003D11048006890F836600F4850F826507D
:103C80002DB94046FCF722FB43202070EAE7012DC6
:103C900005D14046FCF71AFB43202070E2E72F6570
:103CA0004046FCF713FB0020207000BFDAE700005D
:103CB0002100002034000020140E002010B504461E
:103CC0002046FCF7ADFC10BD10B5FCF7AAFC10BDFA
:103CD0002DE9F04707460D464FF0000A0020286006
:103CE0006860FCF7EFFA8246FF2F03D1184800689E
:103CF00090F83670174850F827402CB95046FCF71A
:103D0000E5FA4320BDE8F087012C04D15046FCF7CA
:103D1000DDFA4320F6E7207C00F0010020B9504690
:103D2000FCF7D4FA4520EDE70026D4F80C90D4F83F
:103D300008805046FCF7CAFA00E0761C58F8041BCD
:103D40000029FAD02E60A9EB060068600020D9E7B0
:103D500034000020140E002070B50446101D20F021
:103D600007004FF08076051F28462E60051F284665
:103D70002C60684E051F28462E604FF01236051F36
:103D800028462E604FF00336051F28462E604FF060
:103D90000236051F28462E607610051F28462E6025
:103DA000051F284629604FF01136051F28462E6052
:103DB0004FF01036051F28462E604FF00936051FBC
:103DC00028462E604FF00836051F28462E604FF01B
:103DD0000736051F28462E604FF00636051F284679
:103DE0002E604FF00536051F28462E604FF0043632
:103DF000051F28462E6003F00405002D7ED0F60531
:103E0000051F28462E60444E051F28462E60434E4F
:103E1000051F28462E60424E051F28462E60414E43
:103E2000051F28462E60404E051F28462E603F4E37
:103E3000051F28462E603E4E051F28462E603D4E2B
:103E4000051F28462E603C4E051F28462E603B4E1F
:103E5000051F28462E603A4E051F28462E60394E13
:103E6000051F28462E60384E051F28462E60374E07
:103E7000051F28462E60364E051F28462E604FF03F
:103E80008346051F28462E60324E051F28462E60A9
:103E9000314E051F28462E60304E051F28462E60E5
:103EA0002F4E051F28462E602E4E051F28462E60D9
:103EB0002D4E051F28462E602C4E051F28462E60CD
:103EC0004FF08246051F28462E60294E051F2846C2
:103ED0002E60284E051F28462E60274E051F2846B7
:103EE0002E604FF08146051F28462E60234E051F89
:103EF00028462E603602051F284600E009E02E60A5
:103F00004FF07E56051F28462E600026051F2846C6
:103F10002E6070BDA94B00000000F8410000F04188
:103F20000000E8410000E0410000D8410000D0411D
:103F30000000C8410000C0410000B8410000B0418D
:103F40000000A8410000A0410000984100009041FD
:103F500000008841000070410000604100005041B5
:103F600000004041000030410000204100001041AD
:103F70000000E0400000C0400000A04000004040C1
:103F80002DE9F04105464FF00008FCF79BF980460B
:103F9000FF2D05D12048006890F83650012608E032
:103FA0001D48006890F83600A84201D1012600E0C3
:103FB00000261A4850F825402CB94046FCF786F9EF
:103FC0004820BDE8F081012C04D14046FCF77EF981
:103FD0004320F6E794F838701148C05D94F8391022
:103FE00088430F49C8550846C05D30B994F83A1067
:103FF0000C48007888430B49087094F8340040F06E
:10400000080084F834004046FCF760F9012E01D125
:1040100000F0C6FC0020D4E734000020140E00207D
:10402000260000202500002010B5FCF7FBFA10BD8B
:1040300070B5054600261748007800B170BD1648D7
:10404000007800B1FAE71DB3FCF73CF906461348C7
:10405000006890F838401248005D1049096891F8EE
:10406000391088430E4908550846005D40B90B4891
:10407000006890F83A100B480078884309490870A6
:104080000648006805633046FCF720F900F088FC1C
:1040900000BFD3E7210000202200002034000020D0
:1040A000260000202500002070B50025FCF70AF945
:1040B0000546034804682846FCF708F9204670BD09
:1040C0005400002070B5002600F072F8FCF7FAF8F2
:1040D000064631480068401C2F4908603046FCF70E
:1040E000F5F82E480078012853D12D48007820B1EA
:1040F000012804D0022809D103E001250BE00025A6
:1041000009E0012501202649087004E0012500206E
:104110002349087000BF00BF05B970BD214804687D
:1041200033E0FCF7CFF80646206B50B3206B401EFF
:104130002063206B28BB94F8340000F0370040B1B6
:1041400014F8340F00F0C800207001206070343C77
:1041500002E0002084F8350094F8340000F00800F4
:1041600078B93834A0781049097808430E490870A6
:1041700020780E49085C6178084314F838190B4A16
:10418000505464693046FCF7A1F894F836003F2893
:10419000C7D100BFC1E70000540000202E0000205E
:1041A00044000020400000202500002026000020C0
:1041B00010B5FCF738FA06480088401C044908800E
:1041C0000846008818B10020088000F003F810BDF0
:1041D0000400002010B503480068FFF79FFB044669
:1041E000204610BD64000020F8B54FF42071284827
:1041F00000F078FB4021274800F074FB002514E014
:10420000681C86B205EB8500214901EBC00406EB72
:10421000860001EBC00764202070002084F8250090
:10422000E7601DA02062681C85B20F2DE8D305EB66
:104230008500174901EBC00464202070002084F839
:104240002500E06014A02062002014490860144991
:1042500008801020134908800D4813490860012088
:10426000FFF7BAFA114908600020FFF7B5FA1049C4
:1042700008606A460FA10D480068FEF7D1FF6A4644
:1042800011A10B480068FEF7CBFF00F027F8F8BD3E
:10429000D4220020542700203F0000005C000020B2
:1042A0005A00002058000020680000206000002014
:1042B0006400002075432F4F532D494920546D72DF
:1042C0004C6F636B0000000075432F4F532D49491D
:1042D00020546D725369676E616C000000B587B041
:1042E0000320002180220A4BCDE90132CDE90310E1
:1042F0004FF6FD703D23074A00900748FFF78AFB01
:1043000006AA06A13D20FFF7A1FC07B000BD0000F2
:1043100054250020502700209943000075432F4F5B
:10432000532D494920546D720000000070B50B46B2
:10433000032580F82550012B05D1154EC569366837
:10434000354445610CE085692DB9114EC569366863
:104350003544456104E00E4E856936683544456153
:10436000057D05F007040B4D05EBC4010D682DB963
:1043700008600025C56001258D8006E00A68086098
:10438000C26010618D886D1C8D800025056170BD37
:104390005C0000205427002008B500BF00BF6A461B
:1043A00000211A480068FFF741FAFFF7C5F91848DD
:1043B0000068401C164908600846007800F00708AD
:1043C000144800EBC8073C681AE0E66810496069C9
:1043D0000968884213D1204600F01EF894F82400A2
:1043E000022804D101212046FFF7A0FF02E00220AD
:1043F00084F82500656815B12046A168A8473446B1
:10440000002CE2D1FFF7B8F9C9E7000064000020F2
:104410005C0000205427002030B5057D05F007041E
:104420000D4D05EBC4031D68854205D1C1681960B7
:1044300039B100250D6104E00169C268CA6002B1AA
:104440001161012580F825500025C56005619D8812
:104450006D1E9D8030BD00005427002010B5FBF775
:1044600031FF044606480078401C05490870204684
:10447000FBF72CFFFFF726FEFEF752FF10BD0000F2
:104480002100002001464A1E4FF0E0235A61084AED
:10449000106820F07F4000BF10601A46126942F099
:1044A00005021A611A46126942F002021A61704747
:1044B00020ED00E0704700002DE9F04F05460F4663
:1044C00090469946A87A1C490E5C05F10B00805D68
:1044D00011F800B00BEBC60000F0FF0A174850F8C7
:1044E0002A4000202434E0602760207C20EA080075
:1044F000207484F81190207C243C00F0080068B9F6
:1045000094F83A000E49097808430D4908700D489F
:10451000805D94F8391008430A4988552946204699
:1045200000F012F8206A20B12046216A00F023F83A
:10453000E5615046BDE8F08F78B40000140E00200D
:10454000250000202600002010B590F8382001F149
:104550000B039B5C90F83940A34301F10B04A35477
:1045600023469B5C23B98B7A90F83A40A3438B7225
:104570000023C36110BDF0B5024612F8384F95789C
:104580005678383A0B4618680FE000F10B073F5D8C
:10459000B74300F10B0C0CF8047067463F5D17B988
:1045A000877AAF4387721B1D18680028EDD1F0BDD4
:1045B00010B51B4A1268D061194A126892F8383057
:1045C00000F10B02D25C164B1B6893F839301A438A
:1045D000134B1B6893F8384000F10B031A55827A8D
:1045E0000F4B1B6893F83A301A4382720C4A1268D8
:1045F00092F838100B4A525C094B1B6893F839301B
:104600009A43084B5A541A46525C42B9044A1268FB
:1046100092F83A30044A12789A43034B1A7010BD4C
:104620003400002026000020250000200146002242
:104630008A72002005E0002301F10B021354421C92
:10464000D0B20828F7D370472DE9F041A0211148D6
:1046500000F048F900250DE0681C86B20D4800EB1B
:10466000051400EB06170020207067600AA0E060C8
:10467000681C85B2092DEFD3064800EB0514002015
:104680002070606004A0E060024804490860BDE852
:10469000F0810000740900203F000000100000209D
:1046A00030B501464A6808682AB9CC68606028B10C
:1046B0000025456002E0106000B142608B68002573
:1046C0009D6230BD70B54FF4BD61134800F00AF92A
:1046D000002411E0601C85B204EB44000E4901EB9C
:1046E000C00305EB450001EBC006002018705E60BA
:1046F0000AA05861601C84B23E2CEBD304EB44004A
:10470000054901EBC00300201870586003A05861F0
:1047100008460349086070BD8C0300203F0000007C
:104720000C00002000200B4908600B4908700B4961
:1047300008700B4908700B4908700B4908600B4959
:1047400008600B4908600B4908600B4908700B4969
:104750000870704754000020210000202200002033
:104760002F0000202E000020080000203000002034
:104770001C00002018000020200000205000002015
:1047800000210A4A1170002004E00021084A115457
:10479000411CC8B20828F8D30021064A1170064A05
:1047A0001170064A1160064A11607047250000200A
:1047B0002600002023000020240000203C000020D0
:1047C0003400002070B54FF48F51194800F08AF87A
:1047D0004FF48071174800F085F8002413E0601C46
:1047E000C5B204EB440000EBC400114901EBC00367
:1047F00005EB450000EBC50001EBC0065E610EA0B5
:104800001865601CC4B2332CE9D304EB440000EB00
:10481000C400074901EBC0030020586106A01865D9
:1048200000200649086002480549086070BD000084
:10483000140F0020140E00203F0000004000002054
:104840003800002000B587B00320002180220A4BE9
:10485000CDE90132CDE903104FF6FF703F23074A3F
:1048600000900748FFF7D6F806AA06A13F20FFF7F9
:10487000EDF907B000BD0000140C0020100E002060
:10488000814B000075432F4F532D49492049646CDB
:104890006500000000B587B00320002180220A4B8C
:1048A000CDE90132CDE903104FF6FE703E23074AF1
:1048B00000900748FFF7AEF806AA06A13E20FFF7D2
:1048C000C5F907B000BD0000140A0020100C00203C
:1048D000C14B000075432F4F532D4949205374613C
:1048E0007400000004E0002200F8012B4A1E91B27F
:1048F0000029F8D17047000070B5F0211148FFF78A
:10490000F1FF00240EE004EB44000E4901EBC0056A
:10491000601C00EB400001EBC00068600AA0686109
:10492000601C84B2092CEED304EB4400054901EB72
:10493000C0050020686004A068610846034908605B
:1049400070BD0000F42000203F000000480000205F
:104950002DE9F041F0211048FFF7C4FF00240DE0DD
:10496000601C86B204EB44000B4901EBC00506EB6A
:10497000460001EBC0072F60601C84B2092CEFD306
:1049800004EB4400044901EBC00500202860084600
:1049900002490860BDE8F081E42100204C000020BD
:1049A00010B50024FBF78EFC044613480078F8B9D4
:1049B00012480078E0B900F02DF811481149097843
:1049C00050F82100104908600E4800780F49097816
:1049D00088420DD00C480068C06B401C0A49096829
:1049E000C8630B480068401C09490860FBF785FC58
:1049F0002046FBF76BFC10BD2100002022000020A8
:104A0000140E0020240000203C0000202300002081
:104A1000080000200649074A1278885C0649095CAC
:104A2000034A515C01EBC001044A11707047000059
:104A300078B400002500002026000020240000207B
:104A40002DE9F84F05460F4690469946DDE90AAB39
:104A500000200090FBF736FC009042480468002CD0
:104A60007BD01C3454F8080C3E4908600098FBF7D2
:104A70002DFC44F81C7CA5760020207660766061D1
:104A800044F818BC44F810AC44F8148C0C9824F882
:104A90000C0C24F80A9C0020E077E810207705F041
:104AA0000700E076217F01208840A077E17E012089
:104AB00088406077002020606060E060A060206235
:104AC000A0626062E062206327A060631C3C002655
:104AD00006E0002104F1540040F82610701CC6B214
:104AE000002EF6D02046FEF78FFFFBF7EBFB009081
:104AF0001E4840F825400098FBF7E8FB2046FEF7EB
:104B0000E5FFFBF7DFFB00901948006860610020BB
:104B1000A0611748006810B1154800688461144806
:104B200004603834A07813490978084311490870A3
:104B300020781149085C6178084314F838190E4A46
:104B400050540E480078401C0C4908700098FBF740
:104B5000BDFB0020BDE8F88FFFE70098FBF7B6FB30
:104B60004220F7E7380000203F000000140E00202C
:104B70004000002025000020260000202F000020FB
:104B8000002400BF00BFFBF79DFB044605480068FA
:104B9000401C044908602046FBF798FBFFF752F8D9
:104BA000F1E700003000002010B504480068FFF76E
:104BB00085F8FF20FEF790FF10BD000034000020B4
:104BC00000BF00BF02E0C820FFF732FA1F4800789C
:104BD0000028F8D01E4800686421B0FBF1F01C49A1
:104BE00008600846006828B900201A490870FF20AC
:104BF000FFF7C6F9FBF766FB044615480068642119
:104C00004843154908602046FBF760FB00BFFBF7EF
:104C100059FB0446104800681049086000200E49FE
:104C200008602046FBF752FB0C48006808490968F9
:104C3000B0FBF1F0C0F1640006490870FFF744F8DA
:104C400000F00EF86420FFF7F3F9E0E72000002001
:104C50001800002014000020300000201C0000205C
:104C60007CB5002514E069462846FFF731F8064672
:104C700066B9094850F8254044B1012C06D0D4E962
:104C8000020100EB8100A0640198E064681CC5B2D9
:104C90003F2DE8D97CBD0000140E002002F0010376
:104CA00043B102F002032BB102E0491E002308C009
:104CB0000029FAD17047000010B500231A460E49AA
:104CC0000120FCF79FFE0446002C02DA4FF0FF3073
:104CD00010BD012009498875094888610948C861E3
:104CE0000846FCF70EFD0446002C02DA4FF0FF30B8
:104CF000EEE70020ECE70000801A06000C2E0020F2
:104D0000511E00009926000070B504460D46164657
:104D10000CB9002070BD0DB90020FBE721462A46E2
:104D2000002304E010780870491C521C5B1C21B160
:104D30001AB1107808B1B342F4D301B10AB9002016
:104D4000E8E7B34201D2002008702046E2E710B540
:104D500002460B461146002001E0491C401C19B1D7
:104D60000C780CB19842F8D310BD000010B50121A9
:104D7000C0F30722094B1A4402F0704242F000725D
:104D8000C0F30723054C2344C3F3130342EA431241
:104D9000C3B242EA8302116010BD000000E60F407A
:104DA0000146C1F307200B4A104400F0704040F068
:104DB0000070C1F30722074B1A44C2F3130240EA02
:104DC0004210CAB240EA8200006808B10120704770
:104DD0000020FCE700E30F400146C1F307200B4A27
:104DE000104400F0704040F00070C1F30722074B00
:104DF0001A44C2F3130240EA4210CAB240EA8200E7
:104E0000006808B1012070470020FCE700EA0F406D
:104E100018B50121C0F30722184B1A4402F0704262
:104E200042F00072C0F30723144C2344C3F313036E
:104E300042EA4312C3B242EA8302116000210091A8
:104E400002E00099491C009100991029F9D3002132
:104E5000C0F30722094B1A4402F0704242F000727C
:104E6000C0F30723054C2344C3F3130342EA431260
:104E7000C3B242EA8302116018BD000000E50F4092
:104E800002480349086000BFFEE700000400FA057D
:104E90000CED00E00148006870470000740000203D
:104EA0004FF0E020006920F001004FF0E0210861A0
:104EB00070474FF0E020006920F002004FF0E02141
:104EC00008617047704770B50446FFF7E3FF40F68E
:104ED000B831B0FBF1F000FB04F52846FBF7AEF962
:104EE00070BD704770B5044625686668164828404E
:104EF000B0F1005F27D1300B0003A04223D1FCF7B3
:104F000023FDFFF7D6FFFFF7CBFF4FF0FF300F4930
:104F100008604FF0E021C1F884010C4908310860B5
:104F20004FF0E021C1F88C01FCF716FD0848046041
:104F30002068FBF78AF92068FBF784F90020FBF76B
:104F400087F96068804770BD0000F82F80E100E0BD
:104F500008ED00E010B5042203494FF4BC50FCF703
:104F600017FD0148006810BD7800002001B50098C9
:104F7000012804D00098022801D0002000900422CB
:104F800069464FF4BC50FCF71DFD024900980860CB
:104F900008BD0000780000207FB588B0DDE910452D
:104FA000E0B28DF818004FF47F4104EA01000021BF
:104FB000000A40EA0160C0B28DF819004FF47F0189
:104FC00004EA01000021000C40EA0140C0B28DF863
:104FD0001A004FF07F4104EA01000021000E40EA70
:104FE0000120C0B28DF81B00E8B28DF81C004FF410
:104FF0007F402840000A8DF81D009DF82000000623
:105000009DF8211040EA01409DF8221040EA01205D
:105010009DF82310084305909DF8240000069DF894
:10502000251040EA01409DF8261040EA01209DF835
:105030002710084304909DF8280000069DF82910C9
:1050400040EA01409DF82A1040EA01209DF82B100B
:1050500008430390FFF71EFF064600210398CDE9A1
:10506000000106A93046DDE9043201F0C7F80CB0B2
:1050700070BD000010B50A20FBF7E0F803200949D5
:1050800008600A20FBF7DAF800200749C1F8C002DF
:105090000A20FBF7D3F80020024908600A20FBF73A
:1050A000CDF810BDFCD00F4000E00A4070B50446BA
:1050B000E10901208840C5430A20FBF7BFF803201F
:1050C000084908600A20FBF7B9F80748C0F8C05241
:1050D0000A20FBF7B3F80020024908600A20FBF71A
:1050E000ADF870BDFCD00F4000E00A4000BF03489F
:1050F000806900F001000028F9D1704700F00A40F3
:1051000002E008C8121F08C1002AFAD17047704790
:10511000002001E001C1121F002AFBD170470000EE
:1051200010B5044600F0BAFB0022034941F2883072
:1051300002F02CFB10BD0000215100002DE9FC47BE
:1051400005468846164600BF0DB9BDE8FC8700BF7E
:1051500070892A280EDA4B48408C401C81B249489D
:105160004184C08B401C81B24648C183304602F066
:105170002BF8EAE7776807F10E042088B0F5807F06
:1051800008D12079062805D16079042802D16088E9
:1051900008280ED03B48008D401C81B2394801855B
:1051A000C08B401C81B23748C183304602F00CF8F6
:1051B000CBE73448408B401C81B232484183D4F85D
:1051C0000E000190A0690090281D08B1686810B910
:1051D0004FF0000907E000986968884201D101207A
:1051E00000E000208146B9F1000F01D0012000E06D
:1051F0000220034604F1080201A9284600F094FBAE
:10520000E088B0F5807F03D0B0F5007F2DD12BE092
:10521000B9F1000F26D0022001F0ADF8E080D4F8FB
:105220000E00A0616868C4F80E0000BF00BFA0684F
:10523000C4F81200A089E082A0683860A089B88014
:10524000D8F80000A060B8F80400A081D8F80000E9
:10525000C7F80600B8F80400788131462846AA69E4
:10526000904700E000BF07E006E00648808D401C44
:1052700081B20448818500BF00BF304601F0A4FF21
:1052800000BF62E7000201202DE9FC5F05460F46E2
:105290004FF00A08C1460A260024A34600200190C8
:1052A000B246009000BF5CE004EB84004D4A02EB84
:1052B0008000817C0A2E02D109B966B24FE0002934
:1052C0004DD000BF00BF5DB104EB8402454B03EB42
:1052D000820228685268904202D160B2BDE8FC9F09
:1052E000012928D104EB84003E4A52F8200088B1FD
:1052F00004EB840002EB8000C27C009882422EDB2B
:105300004FFA84FA04EB8400364A02EB8000C07C3A
:10531000009024E004EB8400324A02EB8000C07C61
:1053200058451CDB4FFA84F804EB840002EB800044
:1053300090F813B013E0022911DB04EB8400294A32
:1053400002EB8000C27C0198824208DB4FFA84F9AC
:1053500004EB8400234A02EB8000C07C0190601CB7
:10536000C4B20A2CA0DB07F0020020B90A2E05D136
:1053700007F0010010B94FF0FF30AFE70A2E01DA55
:10538000F4B21AE0B9F10A0F03DA09F0FF0400BF22
:105390000EE0B8F10A0F02DA08F0FF0408E0BAF1F3
:1053A0000A0F02DA0AF0FF0402E04FF0FF3095E73F
:1053B00000BF00BF204600F017F800BF00BF00BFCD
:1053C00000BF35B104EB8401064A02EB8101286875
:1053D0004860002004EB8401024A02EB8101C8749A
:1053E00060B27BE73403012010B5044604EB84006F
:1053F0000C4951F8200060B104EB8401094A52F8CD
:10540000210001F0E1FE002004EB8401054A42F88E
:105410002100002004EB8401024A02EB8101887420
:1054200010BD0000340301202DE9FC4704460F465F
:105430001546A94600BF00BF00BF00BF00BF00BFA8
:105440000E21384601F025FF40B14B484089401CF1
:10545000494948816FF00100BDE8FC872146286872
:1054600000F0A3FC10B1DFF814817DE0287800F093
:10547000F000E02815D101208DF8000000208DF803
:1054800001005E208DF80200687800F07F008DF842
:105490000300A8788DF80400E8788DF80500E84648
:1054A00061E02868A1680840D4E9011211408842EF
:1054B00010D0288880B24FF6A96188420AD004F142
:1054C0000C0020B1E06810B104F10C0902E06FF0AB
:1054D0000300C1E72A48007800EB8000294901EB6E
:1054E0008000807C022818DB2549097801EB8101C6
:1054F000244A02EB8101D9F80000496888420CD1A6
:105500001D48C08D401C81B21B48C1851C480278D3
:105510003946204600F038F89EE700261BE006EBEF
:105520008600184901EB8000807C022811DB06EB25
:105530008601144A02EB8101D9F8000049688842CB
:1055400007D10F490E70F2B23946204600F01CF820
:1055500082E7701C46B20A2EE1DB3A4649462046F5
:1055600000F048F878E700BF434604F12F023946BF
:10557000204600F077F96FE700020120F8B600003E
:10558000120100203403012070B505460E46144672
:1055900000BF00BF04EB8400154901EB8000807C54
:1055A000022817D104EB840001EB8000C07CE428C2
:1055B00010DB04EB84000A4602EB8000011D284644
:1055C00000F03AF930B9032004EB8401084A02EBF9
:1055D0008101887404EB8400054901EB800000F12F
:1055E0000C0305F12F023146284600F03BF970BD4F
:1055F000340301202DE9F05F80460F46164608F17E
:105600002F094FF0FF3A4146386800F0CEFB38B919
:10561000387800F0F000E02802D00FB1386818B9EF
:105620006FF00D00BDE8F09F01213846FFF72CFE1A
:105630000446002C08DA2EB14948808C401C81B207
:10564000474881842046EDE704EB8400454901EB9F
:105650008000807C30B9012004EB8401414A02EBD8
:105660008101887400BF00BF04EB84003D4901EB59
:105670008000807C012800D03EB93946404600F0C9
:10568000DBF882460EB95046CCE700BF00BF04EB02
:105690008400344901EB8000807C02280FDB324912
:1056A0000C7004EB84002F4901EB800000F10C0327
:1056B0004A463146404600F0D5F882464EE004EBBB
:1056C0008400284901EB8000807C012846D14FF0FE
:1056D000000B354608E000BF00BF287B012802D040
:1056E0004FF0010B02E02D68002DF4D100BFBBF19B
:1056F000000F10D029890022032001F0A7FB0546E6
:105700006DB13146284601F0B6FC40B1284601F0A3
:105710005BFD002503E03546284601F059FEA5B1A2
:1057200004EB84000F4951F8200030B104EB8401F0
:105730000C4A52F8210001F047FD04EB84000949AE
:1057400041F820504FF0000A07E00548808C401CCB
:1057500081B2034881844FF0FF3A00BF504661E7B1
:105760000002012034030120120100202DE9F84F2E
:105770000746884691469A46DDF828B000200090FA
:1057800000BF00BF00222A21032001F05FFB054675
:105790004DB92848808C401C81B2264881844FF046
:1057A000FF30BDE8F88F00BF00BF6E6806F10E0441
:1057B0000D9800F0E0FDE08000BF00BFDAF80000C7
:1057C000A060BAF80400A0810B980168C4F8121018
:1057D0008088E082D9F800003060B9F80400B08019
:1057E000D8F80000C6F80600B8F804007081DBF8AD
:1057F0000000C4F80E000C980068A0614FF480709F
:1058000020800820608006202071042060714FF401
:10581000C160B08129463846BA6990470090054872
:10582000008B401C03490883284601F0CDFC00256D
:105830000098B6E7000201207FB504460D4601211D
:10584000064A201D04F12F038DE825000391044A28
:1058500019462046FFF78AFF04B070BDFEB600006F
:10586000F8B600002DE9F04105460E461746984669
:10587000746800BF00BFD8F800002060B8F80400CA
:10588000A0803868C4F80600B88860810820A0812C
:1058900031462846AA699047BDE8F08170B50024DA
:1058A0003DE004EB84001F4901EB8000857C25B3BB
:1058B00004EB840001EB8000C07C401C04EB8401FD
:1058C000184A02EB8101C87404EB8400114601EB15
:1058D0008000C07CF0280DDA04EB840001EB80002E
:1058E000807C01280AD104EB840001EB8000C07C9D
:1058F000022803DB2046FFF777FD0EE004EB84006F
:10590000084901EB8000807C032806D1022004EBCB
:105910008401044A02EB81018874601CC4B20A2C21
:10592000BFDB70BD340301202DE9F04706460D466C
:105930001746984600BF00BF5DB1286848B13146A0
:10594000286800F032FA20B9287800F0F000E0284A
:1059500003D16FF00D00BDE8F08741462846FFF700
:1059600093FC0446002C01DA2046F4E7022004EB05
:1059700084011A4A02EB8101887404EB8400114609
:1059800001EB8000866004EB840001EB8000396845
:10599000C160B9880182002004EB840102EB81011F
:1059A000C87404EB8400114651F8200098B104EB50
:1059B000840051F82090002004EB840142F821007B
:1059C0003B4606F12F0249463046FFF74BFF48465B
:1059D00001F0FAFB00BF0020BDE700003403012006
:1059E0002DE9F04104460E464FF00E0860890E285E
:1059F0000BDC3348008D401C81B231480185C08BDF
:105A0000401C81B22E48C18354E06568AF89287874
:105A100000F00100B0B12878012809D1687888B970
:105A2000A8785E280ED1607B40F01000607309E01A
:105A3000062224492846FAF7F5FC18B9607B40F0A5
:105A400008006073082F03D0B7F5C16F22D114E0AE
:105A500096F8350000F0200000B92BE0C8F10000F6
:105A600001B2204601F015FC10B100BF00BF21E0DB
:105A70003146204600F0C0F918E096F8350000F0F5
:105A8000200000B916E0224606F12F013046FFF74C
:105A900055FB0BE00A48008D401C81B20848018587
:105AA000C08B401C81B20648C18303E000BF0020C8
:105AB000BDE8F081204601F087FB0020F8E70000F8
:105AC00000020120F8B6000070B505460C462246DB
:105AD0000321284600F0F2F870BD00002DE9FE4FCA
:105AE000044689467248B0F84A00401C81B27048AA
:105AF000A0F84A106568287800074FEA9068C8F156
:105B00000001204601F0C5FB10B92089042800D20D
:105B1000B4E0606890F800A0BAF1000F03D0BAF1C9
:105B2000080F7DD100E0A4E001266248007800F073
:105B3000F000E02800D100265E490868494600F0E0
:105B400034F900B1002666B95948B0F85C00401C31
:105B500081B25748A0F85C10204601F035FBBDE843
:105B6000FE8F2089082800D288E0204600F0F2F855
:105B700058B1204601F028FB4D48B0F85000401CB9
:105B800081B24B48A0F85010E9E72421204601F0EB
:105B900080FB48B34146204601F07BFB10B100BFBB
:105BA00000BF77E021890022022001F04FF906466C
:105BB00006B96FE000BF00BF2146304601F05BFA36
:105BC00010B100BF00BF65E07568C8F1000001B208
:105BD000304601F05EFB10B100BF00BF5AE0204626
:105BE00001F0F2FA344608E06FF02301204601F09C
:105BF00050FB10B100BF00BF4CE067682D48006843
:105C0000E8602D4800682861002038707880FF2007
:105C10002872002068812648B0F84800401C00E047
:105C200017E02349A1F848004146204601F031FB26
:105C300008B100BF0CE001200021FF230A46CDE996
:105C4000010900911B49204600F0FEF9064600BFFD
:105C50000FE01748B0F85800401C81B21448A0F873
:105C60005810B0F84E00401C81B21148A0F84E10F8
:105C700000BF00BF204601F0A7FA70E7204601F000
:105C8000A3FA0B48B0F85200401C81B20848A0F8B3
:105C9000521064E7204601F097FA0548B0F85C001E
:105CA000401C81B20248A0F85C1000BF57E700001A
:105CB000000201200C010020080100202DE9FE4314
:105CC00006460F46904600222421012001F0BEF82E
:105CD00005460DB9BDE8FE8300BF00BFD6F80490AD
:105CE0006C68277084F801800020A080E0807168D3
:105CF0006A6802F108001C22FAF756FB0020608057
:105D00006989204600F01CF860800C48B0F8480013
:105D1000401C0A49A1F84800D9F80C000290012063
:105D20000021FF2302AACDE90010284600F068F9FF
:105D3000284601F049FA00BFCCE70000000201202C
:105D400070B504460D462946204600F03BFBC04393
:105D500080B270BD2DE9F04106460024002735468B
:105D600017E06989686800F02DFB0444A0B200EBDD
:105D70001444688900EBD0714910A0EB410139B19E
:105D8000C7F10100C7B2E0B2C4F3072141EA002421
:105D90002D68002DE5D127B1E0B2C4F3072141EA17
:105DA0000024E04380B2BDE8F08118B502460092BD
:105DB000D04300B10AB9012018BD91F8350000F0B8
:105DC000020008B90020F7E74868904201D100209E
:105DD000F2E700988B681840D1E9013423409842DB
:105DE00008D1886822EA00008C68E343984201D118
:105DF0000120E1E70020DFE72DE9F04706460F46E6
:105E00007948408E401C81B2774841867568287871
:105E10000421B1EB201F12D0304601F0D5F97248B1
:105E2000B0F84400401C81B26F48A0F84410C08E06
:105E3000401C81B26C48C1860020BDE8F0872878FC
:105E400000F00F094FF6FF7000EA8909688800F03A
:105E5000B2FA80467089484502DB308940450FDA46
:105E6000304601F0B1F96048408F401C81B25E4875
:105E70004187C08E401C81B25B48C1860020DCE7B0
:105E80004146304601F068FA286958490860E868D8
:105E9000574908604FF0010A3C4600BF94F83500AE
:105EA00000F0010078B1201D68B1606858B14F481A
:105EB00000686168884205D04C4908682146FFF7B0
:105EC00074FF00B10DE0BAF1000F04D04FF0000AEA
:105ED0004848046800E02468BC4200D12468002CD3
:105EE000DCD100BF424908683946FFF75EFF28B998
:105EF0003F48007800F0F000E0280AD1304601F079
:105F000063F93948C08E401C81B23748C1860020F1
:105F100093E724B9304601F057F900208DE7E8886F
:105F20004FF63F71084088B1304601F04DF92E48D8
:105F3000B0F84200401C81B22B48A0F84210C08E3D
:105F4000401C81B22848C186002076E72A480760B5
:105F50002A4805603946304601F08CFAC0BB687AA1
:105F600001280DD0062806D011280ED1394630461A
:105F700004F09EFF2BE03946304602F055F826E04B
:105F800039463046FFF7AAFD21E01849086839462E
:105F9000FFF70BFF50B91548007800F0F000E0283B
:105FA00004D0756002213046FFF78EFD304601F0C7
:105FB0000BF90D48B0F84000401C81B20A48A0F827
:105FC0004010C08E401C81B20748C18600BF00BF90
:105FD000002009490860094908600549086003492B
:105FE000086000BF29E70000000201200C0100202A
:105FF000080100209C000020000100200401002076
:106000002DE9FE4F06460F4615469846DDE90C9AE7
:1060100000BF00BF284600F07DF8041E08D10948E3
:10602000C08F401C81B20748C187201FBDE8FE8F8A
:1060300043462A4639463046CDE9009A029400F09C
:1060400003F8F3E7000201202DE9F84F05460E465C
:1060500017469A46DDF828B0DDF8308000BF00BF53
:10606000002F43D04FF014091421284601F011F9F4
:1060700058B12648B0F84400401C81B22348A0F82B
:1060800044106FF00100BDE8F88F6C6800BF00BFDE
:1060900084F808A00B9860723868206148464FEA7F
:1060A000E97109EB9171C1F3870141F04001217061
:1060B00084F801B0288900F05EF960800020E0805B
:1060C0001348008800F057F9A08011480088401C50
:1060D0000F4908800EB1306818B9D8F80400E060A4
:1060E00001E03068E0600020608103E06C682069B6
:1060F00000906F460548008E401C044908863A46C9
:1061000029464046D8F814309847BCE700020120E1
:106110001001002010B50246144801680FE091F804
:10612000350000F0010048B110688B681840D1E9D3
:1061300001342340984201D1084610BD0968002966
:10614000EDD10B48006830B10948006890F835007F
:1061500000F0010038B90748C08F401C83B20548E1
:10616000C3870020E9E702480068E6E79C000020BA
:10617000A00000200002012070B50025FDF7B6F850
:10618000FAF7A0F8054601211848FBF761F8044624
:1061900004F0805050B11548FBF707F91348FBF79E
:1061A000EEF81248FBF7D5F824F080541CB12146D4
:1061B0000E48FBF70FF804F0005058B10B48FBF7FE
:1061C000E9F806460A48006820B131460748084AFF
:1061D000126890471CB12146064804F0D5FB2846BA
:1061E000FAF774F8FDF79CF870BD000000C00E408F
:1061F0005C010020382F0120704700002DE9FC478A
:1062000004460D4616461F46DDE90A892248FEF778
:10621000ADFD2148FEF7FCFD2048FEF7C1FD30B181
:106220001E48FEF7A3FD1D48FEF7F2FD01E000BF8A
:10623000FEE700BF1848FEF7CFFD0028FAD040F275
:106240000E411748FBF71EF8002004210B46154AA3
:10625000CDE9001021461248FAF768FF00234FF0FD
:1062600008724FF440610E48FAF73EFF2A460021BB
:106270000B48FAF7FCFE0C48C0F800900B4806608B
:106280000B4807600B48C0F8008000210A4804F062
:10629000A7F9BDE8FC870000009C00F0003000F08A
:1062A00000C00E40020000046001002064010020D4
:1062B000680100206C010020D562000010B5044682
:1062C000FFF79AFF00220249012001F05FFA10BD9A
:1062D000BD62000010B586B004461848006878B961
:1062E0001748006800F03AF805901648006800F07A
:1062F00035F804901448006800F030F8039003E08B
:10630000002005900490039010481149002203AB2F
:10631000CDE90021029004AA05A90E4800F0A0FCD6
:106320000C4800F0EBFC0B4800F06DFD00220A4920
:10633000012001F02BFA06B010BD00006001002022
:1063400064010020680100206C01002045A60000C7
:1063500049A90000382F0120BD620000014608064F
:1063600001F47F4240EA022001F47F0240EA122059
:1063700040EA1160704701460806000C40EA11200F
:10638000704710B501F0B0F801F032F900F0CEF826
:1063900000F0B2FA00F09CFC00F013F804F086FD67
:1063A00001F040FE01F05CFA10BD00B5034618464E
:1063B000FFF7D4FF00BD00B502461046FFF7DBFF34
:1063C00000BD7047F8B505460A462B4600200090F0
:1063D000002103F0010636B1002A04DD13F8010B99
:1063E0008DF80100521E1C4603E034F8027B39444C
:1063F000921E012AF9DC002A02DD20788DF80000C7
:10640000BDF80000014488B200EB114188B200EBF6
:10641000114126B1C8B2C1F3072747EA002188B26B
:10642000F8BD000088B006A90FA0FAF709FDF9F73A
:10643000A1FFFCF721FF032000214FF400720E4B57
:10644000CDE90132CDE90310022003460B4A00904A
:106450000B48FDF7DFFA07AA0AA10220FDF7F6FBB9
:10646000FDF788FA00BFFEE7544D34433132395806
:106470004E435A4144000000742F01207037012020
:106480001D050000537461727400000070B505466C
:1064900005B970BD00BF00BF00BF00BF1E48006847
:1064A000854203D31D48006885420FD3002601F0C2
:1064B00063F806461A48B0F89800401C81B21848A4
:1064C000A0F89810304601F08DF8E2E70021154859
:1064D00001F056F8A5F1080400BF00BF00202071AC
:1064E00011480068844201D20F48046020880A499C
:1064F0000988611A411A0A48B0F89200401A81B21C
:106500000748A0F89210204600F070FF054801F0FF
:10651000FDF800BFBDE700008C00002090000020C7
:1065200000020120980000209400002010B500BF58
:1065300000BF174820F003001649086008460468A9
:106540004FF42050208000206080207108460068B1
:1065500000F52050104908600120096808714FF4C7
:1065600020500D49096808800B490968488009488E
:1065700000680A4908604FF420500949A1F89000CA
:106580000121084801F0A8F808B100BF00BF10BD04
:106590002F2E00208C00002090000020940000206E
:1065A00000020120980000202DE9F041054615B9B0
:1065B0000020BDE8F081E81C20F0030085B20C2D1E
:1065C00000DA0C25B5F5205F01DD0020F1E70021A0
:1065D000524800F0D5FF5248008852490988401AB5
:1065E00086B289E04F4800688419207900287CD160
:1065F000218806F10800081AA8427AD3218806F1FA
:106600000800091A05F11400814232D306F108008E
:1066100028441FFA80F84348006800EB0807002070
:106620003871208838807E80A4F800800120207195
:106630003888B0F5205F05D038883A4909680844A1
:10664000A0F8028000BF3848B0F8921005F10800A9
:10665000084481B23448A0F89210B0F89410B0F811
:106660009200814204DA3048B0F89210A0F89410F9
:106670001BE00120207100BF20882A490988611A87
:10668000411A2948B0F89200084481B22648A0F87F
:106690009210B0F89410B0F89200814204DA2248C7
:1066A000B0F89210A0F8941000BF1D480068844212
:1066B00011D11B49086803E001881A4A126888183A
:1066C000017919B1194909688842F5D1144908605E
:1066D00000BF00BF00BF114801F018F800BF00BFA5
:1066E00000BF00BF00BF00BF00E002E004F10800EF
:1066F0005FE70C480068865BC5F52050B0423FF765
:1067000071AF0948B0F89600401C81B20648A0F865
:106710009610024800F0FAFF00204AE79800002097
:10672000940000208C000020000201209000002036
:106730002DE9F05F82460D46E81C20F0030085B28B
:106740000C2D00DA0C25B5F5205F02DD0020BDE838
:10675000F09F00BF00BF4B480068824503D34A4802
:106760000068824511D34FF0000B00F005FF83460F
:106770004648B0F89800401C81B24448A0F89810F0
:10678000584600F02FFF5046E1E7AAF108073D48C0
:106790000088381A1FFA80F93888A0EB09000838F9
:1067A0001FFA80F800BF00BF454501DD0020CEE79D
:1067B000454501D15046CAE70021354800F0E0FECA
:1067C0003888304909684418207950BB208809F17D
:1067D000080129448EB22F490968A14204D12949F0
:1067E000096831442B4A1160264909688C19002137
:1067F00021712080A4F802903E802188B1F5205FAD
:1068000004D021881F4A126811444E801F49B1F8F4
:106810009210A8EB0502891A8AB21C49A1F89220AD
:106820002AE005F11400404526D809F10800284463
:1068300086B214480068841916480068844201D260
:10684000144804600020207138882080A4F8029049
:106850003E802088B0F5205F04D02088094909686F
:10686000084446800948B0F89200A8EB0501401A98
:1068700081B20648A0F89210054800F047FF504644
:1068800065E700008C00002090000020000201203D
:1068900098000020940000202DE9F04104460D46A8
:1068A00000270DB9BDE8F08100BF00BFA5F11C06AF
:1068B00000F062FE074600F0DBF804EB84010C48B0
:1068C00000EB41004088401E81B204EB840208487E
:1068D00000EB42004180074850F824003060054832
:1068E00040F82460384600F07DFE00BFDAE7000083
:1068F0009A0201204056002070B500241CE00021BF
:1069000004EB8402224800EB4200418004EB840245
:106910001F4800EB4200818004EB84021C4800EB1E
:106920004200C1801B4830F8141004EB8402184860
:1069300020F81210601C84B20C2CE0DB164820F00A
:10694000030500241DE00020144941F8240000261E
:1069500010E0124850F824002860104840F82450F5
:106960000F4830F8141005F11C00084400F1100520
:10697000701C86B2074830F81400B042E9DC601C95
:1069800084B20C2CDFDB00F033F900F071F870BD3D
:106990009A02012090B50000735600204056002056
:1069A00078B500002DE9F04104460E4617464FF039
:1069B000000800BF0C2C02DB0020BDE8F08100BF06
:1069C00000F0DAFD804600F053F8274850F82450D4
:1069D000ADB32549286841F82400002028606E6086
:1069E000AF6000BF04EB8401204800EB4100408809
:1069F000401C81B204EB84021C4800EB4200418041
:106A000004EB8401194800EB4100818804EB840207
:106A1000164800EB4200408881420BDA04EB840107
:106A2000124800EB4100418804EB84020F4800EB60
:106A30004200818000BF00BF00BF1C350EE0FFE7B1
:106A400004EB8401094800EB4100C088401C81B27E
:106A500004EB8402054800EB4200C180404600F090
:106A6000C1FD2846A9E70000405600209A020120F7
:106A700070B51F4820F00305002417E000BF002672
:106A80000DE02146284600F039F81A4830F8141075
:106A900005F11C00084400F11005701C86B2164870
:106AA00030F81400B042ECDC601C84B20C2CE5DB46
:106AB0000F4820F00305002417E000BF00260DE07A
:106AC0002146284600F05AF80A4830F8141005F11B
:106AD0001C00084400F11005701C86B2064830F80E
:106AE0001400B042ECDC601C84B20C2CE5DB70BD01
:106AF0007356002078B5000090B50000F0B5A1B045
:106B000006460C461A4830F8141006F11C000F18FF
:106B1000002529E0785DCD2824D08022154901A8E0
:106B2000F9F742FC14A0006800900A2C0ADB0A2046
:106B300094FBF0F03030C0B28DF80000694601A837
:106B4000F9F756FC0A2094FBF0F100FB11403030BD
:106B5000C0B28DF80000694601A8F9F749FC00BFF2
:106B600000BF00BF681C85B2102DD3DB21B0F0BD83
:106B700078B50000A8B5000030000000F0B5A1B065
:106B800006460C4606F10C07002529E0785DCD2865
:106B900024D08022144901A8F9F706FC13A000684C
:106BA00000900A2C0ADB0A2094FBF0F03030C0B2CF
:106BB0008DF80000694601A8F9F71AFC0A2094FB39
:106BC000F0F100FB11403030C0B28DF80000694692
:106BD00001A8F9F70DFC00BF00BF00BF681C85B21B
:106BE000102DD3DB21B0F0BD28B60000300000002E
:106BF0002DE9F041174820F00305002425E000BFEF
:106C000000261BE005F10C07CD2210213846F9F7CC
:106C1000DDFB114830F8141005F11C000F18CD22CF
:106C200010213846F9F7D2FB0B4830F8141005F163
:106C30001C00084400F11005701C86B2074830F8AB
:106C40001400B042DEDC601C84B20C2CD7DBBDE843
:106C5000F08100007356002078B5000090B5000068
:106C60002DE9F04704460D4616461F46DDE909A901
:106C7000DDF8208000BF00BF00206060A060E06001
:106C800084F83500E0612062C4F828800E4800785E
:106C900084F838000C480078401C0B490870C4F890
:106CA00010903B4632462946204600F012F8204616
:106CB000D04710B10020BDE8F0870448006820608C
:106CC000024804602046F6E7A40000209C00002053
:106CD00070472DE9F04106460F4614461D463946D9
:106CE000304600F017F82146304600F086F8294675
:106CF000304600F009F8BDE8F08100000149086065
:106D000070470000A000002009B9002200E00A68D6
:106D1000C26070472DE9F04107460C4654B3206825
:106D20007968884201D1012000E0002010BB15489D
:106D300006680BE030687968884206D1D6F80C8086
:106D4000304600F065FE464600E0F668002EF1D1C0
:106D50000D4805680CE055B1286840B1286879688D
:106D6000884204D10CB9002000E020682860ED685A
:106D7000002DF0D10CB9002000E020687860BDE85B
:106D8000F0810000BC000020B800002010B50446CF
:106D900094F8350000F0100060B194F8350020F050
:106DA000100084F8350000BF206A10B12046216A27
:106DB000884700BF10BD10B5044694F8350000F0B8
:106DC0001000C8B914F8350F40F01000207014F806
:106DD000350900F0010040B194F8350000F02000C2
:106DE00018B1211D2046FEF727FD00BF206A10B113
:106DF0002046216A884700BF10BD09B9002200E083
:106E00000A688260704710B5044694F8350000F0B7
:106E10000100D0B994F8350040F0010084F8350045
:106E200000BFE06910B12046E169884700BF94F8CF
:106E3000350000F0100040B194F8350000F020005B
:106E400018B1211D2046FEF7F7FC10BD2DE9F05FBB
:106E500083460F469046BBF1000F09D0BBF1010FEE
:106E600008D0BBF1020F07D0BBF1030F08D105E03A
:106E700038260AE0242608E0102606E0002604E072
:106E800000BF00BF0020BDE8F09F00BFB8F1000FB9
:106E900078D0B8F1010F72D0B8F1020F70D0B8F10C
:106EA000030F6ED1EF2256A10B20FFF77BFD0446A6
:106EB0001CB900F02DFA0020E5E784F80C800020D2
:106EC000206006F110002044C01C20F00300606028
:106ED00000BF00BF2781F01C20F0030040F2EC51FE
:106EE000081AB84201DD384605E0F01C20F0030026
:106EF00040F2EC51081A608100BF00BF00BF00BF24
:106F00000120E081A2466089A7EB000932E04FF43E
:106F100088723BA10B20FFF745FD054635B900F00F
:106F2000F7F9204600F050F90020ACE785F80C8016
:106F3000002068732860CAF8005000BF00BFA5F8A1
:106F400008901FFA89F040F2EC51884202DA1FFAE9
:106F500089F001E040F2EC50688105F110006860B2
:106F600000BF00BF00BF00BF0120E8816889A9EB16
:106F70000009AA46B9F1000FC9DC39E002E020E0BF
:106F800020E031E006F1130121F00302F91C21F0A9
:106F90000301114488B2FFF707FB04460CB9002037
:106FA00071E704F110003044C01C20F00300606061
:106FB000278167810020206084F80C8000BF00BF1B
:106FC00016E000BF4FF4A3720DA10A20FFF7EAFC00
:106FD00004460CB9002056E70020606027816781D5
:106FE000206084F80C8003E000BF00BF00204AE767
:106FF00000BF0120E08100206073204643E70000CD
:107000002E2E5C5372635C5573725C4472697665B4
:10701000725C55704472697665725C6C7769705CFD
:10702000636F72655C706275662E630010B5024610
:1070300000BF02B101B910BD00BF104604E00389D2
:107040000C892344038100680368002BF7D100BF3B
:1070500000BF00BF00BF03890C8923440381016086
:1070600000BFE8E70146002002E0421CD0B20968F8
:107070000029FAD170472DE9F04105460C4600265B
:10708000002700BF25B11CB128892189884203DA75
:107090006FF00D00BDE8F08100BF00BF6889801B64
:1070A0006189C91B884204DB6089C01B1FFA80F814
:1070B00003E06889801B1FFA80F86268D1196A684A
:1070C00090194246F9F770F906EB080086B207EB13
:1070D000080087B200BF00BF00BF00BF6089B84290
:1070E00001DC002724686889B04208D100262D6899
:1070F00000BF1DB914B16FF00D00CBE700BF54B154
:1071000060892189884206D100BF206810B16FF0E4
:107110000500BFE700BF55B168892989884206D1BB
:1071200000BF286810B16FF00500B3E700BF002C66
:10713000B4D10020AEE72DE9F05F804689461646BF
:107140001D464FF0000B00BFB8F1000F02D1002028
:10715000BDE8F09F00BF00BFB9F1000F01D10020D2
:10716000F6E700BF4FF0000AB8F1000F02D0B9F106
:10717000000F01D10020EBE7444620E035B16089E3
:10718000A84203DC6089281A85B217E06089401B99
:1071900087B2B74200DD37466268511909EB0A0031
:1071A0003A46F9F701F90BEB07001FFA80FB0AEBEF
:1071B00007001FFA80FAF01B86B2002524680EB182
:1071C000002CDBD15846C3E72DE9F047044624B92B
:1071D00000BF00BF0020BDE8F08700BF00BF002651
:1071E0002DE04FF0000900F0C7F9814600BF00BF55
:1071F000E089401E1FFA80F8A4F80E80484600F08F
:10720000F1F9B8F1000F18D12768257B032D04D1BF
:1072100021460B20FFF740FB0BE0012D01D0022D92
:1072200004D121460A20FFF737FB02E02046FFF792
:107230002DF9701CC6B23C4600E0002400BF002CB3
:10724000CFD13046C7E7000070B5002500F094F9B3
:10725000054600200A490870284600F0C3F909488D
:10726000046808E0606F28B1606F02F068FE0020DB
:10727000606770BDE468002CF4D100BFF9E700003E
:10728000A5000020BC00002010B50446FFF7DCFF7D
:1072900010BD70B5024600BF00BF01B10AB90020A1
:1072A00070BD002908DA484284B200BF5089A0426C
:1072B00001DA0120F4E700E08CB2137B55680BB1D2
:1072C000032B0AD15068401A506002F11000566832
:1072D000864215D255600120E2E7022B01D0012B36
:1072E0000AD1002906DA5089A04203DB5068401A0F
:1072F000506005E00120D3E700BF00BF0120CFE7C9
:107300005089084450811089084410810020C7E743
:1073100070B5002500F030F905460D4804780120CD
:107320000B490870284600F05DF984B900BF0022BF
:107330001146084803F00CF940B100F01DF905466C
:10734000002003490870284600F04CF900BF70BDCA
:10735000A5000020897200002DE9F04106460F4685
:1073600000BF00BF00BF00BF3089B84201DCBDE8EC
:10737000F0813089A7EB00083D4634460AE0608979
:10738000281A85B200BF00BF2089404420812468AC
:1073900000BF00BF6089A842F1DB207B60B9608933
:1073A000A84209D0A088001B284481B22046FFF7DC
:1073B000BFF9044600BF00BF658160892081206855
:1073C00010B12068FFF700FF0020206000BFCEE76B
:1073D00070B50446002544B100F0CEF80546E089BA
:1073E000401CE081284600F0FDF870BD30B500BFBC
:1073F00000BF00BF00BF00BF00BF00BF00BF0388C9
:10740000194C24681919884215D00B799BB9174B70
:107410001B6899420FD0164B1B688B4201D1144B4D
:1074200018600B880380104B1B88C31A0C880E4D04
:107430002D682C44638043880B4C24681A198242BF
:1074400011D013797BB90A4B1B68834201D1084BD9
:107450001A6003881380044B1B88D31A0488024DDA
:107460002D682C44638030BD8C00002090000020EB
:10747000940000202DE9F04705468A460027D5F8FC
:10748000048098F809900026144804681FE0207CC6
:1074900048451AD134B1206820B1114920680968E3
:1074A000884212D1606980B10E4B2A462146D4E948
:1074B00005C0E04748B10025012736B1E068F0601B
:1074C00006480068E060054804602646E4680FB995
:1074D000002CDCD13846BDE8F0870000A800002071
:1074E0000C01002008010020704700002DE9F84F32
:1074F00081460E461446D9F800A04CB14FF47A707C
:1075000060434FF47A71B0FBF1F717B9012700E03F
:107510000027FCF7C9FD0446B9B26A46DAF8000054
:10752000FCF70EF880463EB11248804502D100209B
:10753000306001E0C6F800809DF800000A2802D102
:107540004FF0FF3413E000BF00BFFCF7ADFD054670
:10755000A54201D92D1B02E0C4F1FF3005444FF4D0
:107560007A7068434FF47A71B0FBF1F0441C204606
:10757000BDE8F88F1C01002010B5F8F7A3FE10BD80
:10758000F8B507460C464CB14FF47A7060434FF49F
:107590007A71B0FBF1F616B9012600E00026FCF77F
:1075A00083FD0446B1B26A463868FCF73FF99DF89E
:1075B00000000A2802D14FF0FF3411E0FCF774FDFF
:1075C0000546A54201D32D1B02E0C4F1FF3005445E
:1075D0004FF47A7068434FF47A71B0FBF1F0441CB9
:1075E0002046F8BD10B504462046F8F76FFE10BDE2
:1075F00008B56B46542214210248FBF7D9FE024914
:10760000086008BDFC0301201401002038B50446C1
:107610000D46142D00DD142569460E480068FBF761
:1076200005FF20609DF8000080B9A9B22268101DF6
:10763000FBF736FF216808602068006808B1002069
:1076400038BD214603480068FBF70FFF4FF0FF30BD
:10765000F6E700001401002070B504460D4605B998
:10766000044D00BF216808682946FBF7FBFF00288E
:10767000F8D170BD1C01002070B505460E4606B954
:10768000064E296808683146FBF7ECFF04460CB942
:10769000002070BD4FF0FF30FBE700001C01002010
:1076A000F0B585B00446256814216846F8F795FEC4
:1076B00069462868FCF70FF80646022E07DABDF87F
:1076C0000400BDF80610884201DA012000E0002025
:1076D0000746384605B0F0BD38B504460D46284685
:1076E000FCF77AF82060206810B94FF0FF3038BD01
:1076F0006A4603A12068FBF793FD0020F7E700002E
:107700004C5749502053656D0000000010B50446E9
:107710002068FCF703F910BD2DE9F04385B08046E1
:107720000D4616461F460C9C4FF0000900BF00BFD7
:1077300010A14046F8F768FEB0B9F8F7C3FD8146DE
:10774000032000214FF400620E4BCDE90132CDE958
:107750000310A0B2E3B20C4A00902846FCF75AF995
:107760004846F8F7B3FD00E00024E0B205B0BDE8FC
:10777000F083000074637069705F7468726561649F
:10778000000000008C0A0120882A01202DE9F04128
:1077900006460F46904640F20F1224A10920FFF73B
:1077A00001F904461CB900BF00BFBDE8F08100200C
:1077B0002060A760C4F80C8066602848006810B993
:1077C00026480460F1E7254800684068B0420CD9BB
:1077D000224800684068801B2049096848601F48AB
:1077E000006820601D4804601DE01C48056817E023
:1077F00060686968401A6060286820B1286840683D
:10780000616888420BD9286828B128684068616897
:10781000401A29684860286820602C6002E02D68C2
:10782000002DE5D100BF00BFBFE700002E2E5C5346
:1078300072635C5573725C4472697665725C5570F4
:107840004472697665725C6C7769705C636F7265AF
:107850005C74696D6572732E63000000F000002097
:1078600010B50022024941F28830FFF78FFF10BDAA
:10787000215100002DE9F0478046894600BF22488B
:10788000006830B9002249464046FFF72FFE054602
:1078900037E01D480068406840B11B480068494611
:1078A00042684046FFF722FE054601E04FF0FF35F3
:1078B000681CA8B914480468134920680860A668C1
:1078C000E76821460920FEF7E7FF46B100210F488F
:1078D000FFF756FE3846B0470C48FFF717FFCEE7D4
:1078E000094800684068A84207D90748006840680E
:1078F000401B05490968486003E000200249096807
:107900004860BDE8F0870000F000002088000020FB
:107910002DE9F04106460F461448006808B9BDE855
:10792000F0811248046800251BE0A068B04216D11F
:10793000E068B84213D11DB90C492068086001E025
:1079400020682860206828B1206840686168084481
:107950002168486021460920FEF79EFFDFE72546A3
:107960002468002CE1D100BFD9E70000F00000201E
:107970002DE9FC4704460E4600BF00BF207E0A28C2
:1079800008D121461F4801F053F921460220FEF795
:1079900083FF34E0276DD4F82880D4F88C50D4F8D5
:1079A000109000BF2146184801F042F90120174904
:1079B000087000BF206F10B1206F02F0C0FAE06EB7
:1079C00010B1E06E02F0BBFA606F10B1606F02F0B0
:1079D000B6FA4EB1A08B618B231D2246CDE9001073
:1079E0004146384602F02AFA21460220FEF754FFAB
:1079F00000BF1DB16FF009014846A84700BFBDE8B0
:107A0000FC870000C0000020BC000020C80000204F
:107A100010B5044601212046FFF7AAFF10BD000063
:107A200070B5064640F2035239A10220FEF7BAFFB4
:107A30000446002C25D100F0D9FD40F2095234A1B2
:107A40000220FEF7AFFF044694B9304600F0A4FDD3
:107A500040F20F522EA10220FEF7A4FF04463CB1D3
:107A60003648B0F8B400401E81B23448A0F8B410D3
:107A70003CB13248B0F8B400401E81B22F48A0F8A3
:107A8000B410002C41D0A0212046F8F7A6FC1834F1
:107A9000667041F2D060A4F84E000020A4F85000B7
:107AA00042F23820A082E082002004F80F0CFF2070
:107AB00004F80E0C4FF40670E0830620A085002029
:107AC000208506206085C01FA0830120A08600F0CD
:107AD0004DFE05462564A563256365641848006866
:107AE000E0601848007860720020E0711648A066D7
:107AF00040F6B830A0674FF4FA60E0670620C4F89B
:107B00008000002084F88600183C204670BD0000EC
:107B10002E2E5C5372635C5573725C447269766599
:107B2000725C55704472697665725C6C7769705CE2
:107B3000636F72655C7463702E6300000002012045
:107B4000B0000020CA000020C59C000010B504460B
:107B5000207E012803D0A07F40F01000A0770121F3
:107B6000204600F001F810BD7CB504460E46002EFC
:107B70005BD0207E042802D0207E072855D1A06F3C
:107B800020B9A08D42F2382188424ED000BF00BFFC
:107B9000A08B618BCDE90010231D2246A16A206DC8
:107BA00002F04CF9204601F01FF800BF00BF5A4810
:107BB0000068A04205D158480068C068564908606E
:107BC00018E055480068554908600EE053480068C1
:107BD000C068A04204D15149E0680968C86008E063
:107BE0004E480068C0684D4908604C48006800284D
:107BF000ECD100BF0020E06000BF012048490870C0
:107C000000BF207E04280AD10A20207600BF454804
:107C10000068E0604348046002F092FB03E0214604
:107C20000220FEF739FE00207CBD207E082868D2A5
:107C3000DFE800F004343F4F5767675F0025608B33
:107C400030B300BF38480068A04205D1364800680C
:107C5000C0683549086018E0334800682F4908605B
:107C60000EE02E480068C068A04204D12B49E068AD
:107C70000968C86008E029480068C06827490860AA
:107C8000264800680028ECD100BF0020E06000BF5B
:107C900021460220FEF700FE002435E000252146A3
:107CA000224800F0C5FF21460320FEF7F5FD002421
:107CB0002AE0002500BF2146174800F0B9FF012047
:107CC0001749087000BF21460220FEF7E5FD002499
:107CD0001AE0204602F066F905460DB90520207627
:107CE00012E0204602F05EF905460DB90520207627
:107CF0000AE0204602F056F905460DB90920207623
:107D000002E00025002400BF00BF1CB115B92046C9
:107D100000F082FD284687E7BC000020C400002058
:107D2000C8000020C0000020B4000020B8000020DF
:107D30002DE9F05F07460E4691469A46DDF8288009
:107D400008F0010008B1042000E0002008F0020162
:107D500009B10C2100E000214518A42224A104202F
:107D6000FEF720FE041E05D13046FFF72DFA002055
:107D7000BDE8F09F84F80A800020206066603089AA
:107D8000401B208114213046FFF783FA60B124485C
:107D9000B0F88C00401C81B22148A0F88C1020461D
:107DA00002F0C0F80020E3E760684068E060788B8C
:107DB000FEF7E1FAE1680880B88BFEF7DCFAE168CB
:107DC00048805046FEF7CAFAE1684860AB46E917BA
:107DD00005EB91718910491D49EA013188B2FEF71E
:107DE000CAFAE16888810020E16848822046BFE73E
:107DF0002E2E5C5372635C5573725C4472697665B7
:107E0000725C55704472697665725C6C7769705CFF
:107E1000636F72655C7463705F6F75742E630000CE
:107E2000000201202DE9F04105460E463046FEF7DE
:107E300071F9044654B1A08D40B1A08D283887B2A5
:107E4000BD4201DA284600E0384605462846BDE82E
:107E5000F08100002DE9F84304460D460027B8469E
:107E600000BF00BFB4F86800102805DAB4F8680055
:107E70004FF6FC7188420FD94A48B0F88400401C84
:107E800081B24848A0F88410A07F40F08000A0771D
:107E90004FF0FF30BDE8F88305F0020000B1012784
:107EA00007F0010008B1042000E0002007F0020103
:107EB00009B10C2100E0002100EB0108B4F86600D4
:107EC00050B93848B0F88400401C81B23548A0F859
:107ED00084104FF0FF30DDE7002241461046FEF7E8
:107EE000B5FFB0F100090ED1A07F40F08000A0776F
:107EF0002C48B0F88400401C81B22A48A0F88410B5
:107F00004FF0FF30C6E700BF00BF00972A46494642
:107F10002046E36DFFF70CFF061E0DD1A07F40F059
:107F20008000A0771F48B0F88400401C81B21D4833
:107F3000A0F88410701EADE700BF00BF00BF00BFF7
:107F4000E06E08B9E66607E0E06E00E000680168F0
:107F50000029FBD1066000BF0020A4F86A0005F0EC
:107F6000020010B905F0010038B1E06D401CE06579
:107F7000B4F86600401EA4F8660005F0010018B1D0
:107F8000A07F40F02000A0777068FFF76BF834F80E
:107F9000681F0844208034F8680908B100BF00BF9A
:107FA000002077E70002012070B51B480078401CD4
:107FB0001949087000BF1948046829E094F82100A5
:107FC00015490978884223D01348007884F82100A5
:107FD000A07F00F0010060B100BFA07F40F0020070
:107FE000A07700BF204600F017FCA07F20F0030020
:107FF000A077E568A06F48B10020094908702046C5
:1080000001F026F90648007800B1D4E72C4600BFFD
:10801000002CD3D170BD0000CA000020BC0000209D
:10802000C8000020704700002DE9FC4706468A463C
:10803000FB48B0F87A00401C81B2F948A0F87A10E9
:10804000F84970680860F74871680068007800F0C7
:108050000F0001EB8000F4490860F24800680078E6
:108060000007800E41423046FFF713F910B93089FE
:10807000142808D2EA48B0F88200401C81B2E848CF
:10808000A0F882103BE2E94908685146FDF78DFEF1
:1080900028B9E648007800F0F000E02808D1E04870
:1080A000B0F88800401C81B2DD48A0F8881026E2B4
:1080B000DD4909688889FEF77EF94FEA20394FEAE1
:1080C000890041423046FFF7E4F840B1D448B0F8A7
:1080D0008200401C81B2D248A0F882100FE2D2493F
:1080E00009680888FEF767F9CF4909680880CE4912
:1080F00009684888FEF75FF9CB4909684880CA4992
:1081000009684868FEF751F9C74909684860C849D5
:108110000860C54909688868FEF747F9C2490968D7
:108120008860C4490860C0490968C889FEF743F9F6
:10813000BD490968C881BC4909688889FEF73BF9CF
:1081400000F03F00BC4908703089097801F0030154
:1081500009B1012100E000210844B8490880002746
:10816000B74804682AE000BF00BF00BF00BF00BFDF
:1081700000BFA08BAC490968098888421CD1608B7C
:10818000A94909684988884216D1AE4960680968DA
:10819000884211D1A5492068096888420CD100BFE6
:1081A00000BF37B1E068F860A5480068E060A44807
:1081B000046000BF00BF03E02746E468002CD2D172
:1081C00000BF002C4DD1A048046820E000BF00BFD4
:1081D000A08B954909680988884217D1608B92491C
:1081E00009684988884211D19649606809688842BF
:1081F0000CD18E4920680968884207D1204602F0D8
:10820000BBF83046FEF7E0FFBDE8FC87E468002CD1
:10821000DCD100278D48056810E0688B8249096829
:108220004988884208D1814928680968884202D073
:108230000DB1286800B903E02F46ED68002DECD1A0
:1082400000BF75B137B1E868F86080480068E86041
:108250007E480560284600F0E7F93046FEF7B4FF97
:10826000D2E7002C7ED0002079490860308908814F
:10827000084646606C480068C86000207549086080
:10828000754908706C48007800F0080018B1707BE0
:1082900040F001007073A06F98B1204600F0D8FF45
:1082A0000A3028B1A06F60B164480088002808DD5A
:1082B0005B48B0F87E00401C81B25948A0F87E109F
:1082C000DDE066480460204600F0FCFC804608F1D2
:1082D0000A00002817D06048007800F0080098B124
:1082E00000BFD4F88C0028B16FF00A01D4F88C20BC
:1082F0002069904700BF2146514800F099FC214673
:108300000220FEF7C9FAB9E05348007800F01000E7
:10831000B8B1A07F00F0100050B900BFD4F88C00B5
:1083200028B16FF00B01D4F88C202069904700BF72
:108330002146434800F07CFC21460220FEF7ACFABF
:108340009CE04FF00008B4F86400002812DD00BF84
:10835000E06F40B1B4F864202146E36F206998478C
:10836000804602E09BE04FF0000800BF08F10A00E1
:1083700000B984E03748006870B300BF00BFA07F39
:1083800000F0100038B133480068FEF71DFF2046AA
:10839000FFF73EFB73E000BFD4F8800048B1002334
:1083A0002C49D4F880C020690A682146E0478046FD
:1083B00007E00023274821460268184601F082FCA6
:1083C000804600BF08F10A0000B958E0B8F1000F7C
:1083D00002D020480068A0671F48007800F0200005
:1083E000E8B1A06F30B1A06F407B40F02000A16FDA
:1083F00048733DE0A08D42F23821884202D0A08D22
:10840000401CA08500BFD4F8800048B300231A4662
:108410002146D4F880C02069E047804623E027E069
:1084200000020120D4000020D00000200C01002018
:10843000D8000020DC000020E0000020E200002046
:10844000BC00002008010020C0000020B80000206F
:1084500024030120E8000020E4000020EC000020BC
:10846000FFE74FF0000800BF08F10A0000B906E07E
:10847000002029490860204600F0CEF900BF002006
:10848000254908602549086025484068A0B324496B
:108490004868FEF799FE0020214948602CE02149F8
:1084A00009688889FDF787FF00F0040008BB1E48B3
:1084B000B0F88800401C81B21B48A0F88810B0F8C2
:1084C0007E00401C81B21848A0F87E101548006854
:1084D0000088144909684988CDE9001013480068EC
:1084E000134A12888118134B134A1448006801F08C
:1084F000A5FC3046FEF768FE00BF00BF84E60A48D0
:10850000B0F87E00401C81B20748A0F87E103046CB
:10851000FEF75AFE00BF77E6EC000020E8000020DE
:1085200024030120D000002000020120D8000020F8
:10853000E2000020080100200C010020DC000020E7
:108540002DE9FC410446216D481EFDF707FF074653
:108550003B4600221146204600F03EFA05460DB982
:10856000BDE8FC816E680B48B0F87800401C0949F2
:10857000A1F8780006200021CDE90010A37A221D81
:1085800021462846FDF73CFD2846FEF71DFE00BFAC
:10859000E6E70000000201202DE9F04106464FF019
:1085A0007F08002700250F48046813E0607EB04272
:1085B0000FDC607E40450CDC0B49606A0968081AD4
:1085C000B84206D30849606A09680F1A254694F82C
:1085D0001980E468002CE9D115B12846FFF718FA94
:1085E000BDE8F081BC000020B000002070B500267E
:1085F00000250B4804680BE00A49606A0968081AFC
:10860000B04204D30749606A09680E1A2546E46837
:10861000002CF1D115B12846FFF7FAF970BD000022
:10862000C0000020B00000207CB505464548007819
:1086300000F0040008B100207CBD4248007800F042
:10864000100098B14048006800883F49096849888F
:10865000CDE900103D4800683D4A128881183D4B25
:108660003D4A3E48006801F0E9FB69E03548007882
:1086700000F00200002863D0687EFFF7D1F90446BD
:1086800054B93748B0F88400401C81B23448A0F88F
:1086900084104FF0FF30CFE72F4800682060688BD0
:1086A00060832C4800686060274800680088A083C9
:1086B0000320207625480068401CA062A06A206341
:1086C00021480068C089A4F860001F480068C0897C
:1086D000A4F86200B4F86000A4F84E001B480068DB
:1086E000401E60652869206168696061287A00F031
:1086F0008C00207200BF00BF1A480068E060194873
:10870000046001F01DFE00BF01201749087000BF82
:10871000204600F00DFAE08E211DFFF783FBE08676
:1087200012212046FFF796FB06462EB10021204677
:10873000FFF71EF930467FE7204600F06DF87BE733
:10874000002079E7E0000020D0000020D8000020C1
:10875000E2000020080100200C010020DC000020C5
:1087600000020120BC000020C8000020044800686E
:1087700004490968084402490860084600687047CF
:10878000CC000020B000002070B505460C46E9681A
:108790008889FDF710FE00F0010020B1204601F0AD
:1087A000CEFB002433E013E0E1688889FDF703FE87
:1087B00000F0010038B10120FDF7DDFDE96889898D
:1087C0000843E968888126462468304601F0AAFB00
:1087D0004CB1E06840682189084429890D4A126833
:1087E0001144081AE0D594B128890A490968084457
:1087F000E1684968401A002809DDE0688088054979
:108800000988401A288129896868FEF7A5FD2C602F
:1088100070BD0000D80000202DE9F047044600BFDD
:1088200000BF6C480068A04202D10020BDE8F0877C
:10883000B4F86000B4F84C10884202DAB4F8600072
:1088400001E0B4F84C008146E56EA07F00F0020024
:1088500070B14DB1E9684868FDF7A7FDA16C401AF9
:1088600029890844484503D9204601F074FBDDE717
:10887000266F26B100E0366830680028FBD191E011
:1088800000BFE9688889FDF796FD00BF206FA0B1A1
:10889000A07F00F0440080B9E06E38B1E06E00685F
:1088A00058B9E06E0089E18E884206DAB4F86600B5
:1088B00018B1B4F86800102801DB012000E00020A6
:1088C00020B9A07F00F0A00000B977E02868E0663A
:1088D000207E02280BD01020FDF74DFDE968898924
:1088E0000843E9688881A07F20F00300A077214633
:1088F000284600F0ADF8E9684868FDF756FD0746E0
:10890000E9688889FDF757FD00F0030008B10120F0
:1089100000E000202989084407EB0008206DB0EB37
:10892000080001D5C4F85080E9688889FDF743FD47
:1089300000F0030008B1012000E00020298908446C
:1089400000282BDD00202860206F10B925672E46F7
:1089500027E0E9684868FDF728FD0746F1684868A0
:10896000FDF723FD381A16D504F1700700E03F68C3
:10897000386860B13968C9684868FDF716FD8246F5
:10898000E9684868FDF711FDBAEB0000EFD43868DC
:1089900028603D6005E03560366802E0284601F059
:1089A000C1FAE56E55B1E9684868FDF7FEFCA16CB7
:1089B000401A2989084448457FF662AF00BFE06E3F
:1089C00010B90020A4F86A00A07F20F08000A077F2
:1089D00000202BE7EC0000202DE9F04705460E466D
:1089E0009046994606F11400404481B200220120CD
:1089F000FEF72CFA074647B300BF00BF7C68688BC0
:108A0000FDF7B9FC2080A88BFDF7B5FC6080C4F8A9
:108A10000490A86AFDF7A2FCA060B246F11706EB2D
:108A200091718910491D102242EA013188B2FDF787
:108A3000A2FCA081E88DFDF79EFCE0810020208251
:108A40006082E98DA86A084428633846BDE8F0874B
:108A50002DE9FC4705460C46A06AFDF77FFCE96856
:108A60008860E08DFDF787FCE968C881E18DA06A28
:108A700008442063E86800F11408A87A00F00100B7
:108A800070B1211D40F2B450FFF7CCF9814649F096
:108A90000170FDF763FCC8F8000008F1040800BF8E
:108AA000B4F93400401C08B90020A0860CB120683D
:108AB00040B9201DFDF72EFB06460EB9BDE8FC8728
:108AC00070682060A06B38B917480068A063E96837
:108AD0004868FDF76AFCE063A88969688988401ADC
:108AE00087B268684089C01B6968488168680089E6
:108AF000C01B696808816968E86848600020E96807
:108B000008820A48B0F87800401C0849A1F87800AB
:108B10000621607ACDE90001A37A221D214668680A
:108B2000FDF76EFA00BFC9E7B00000200002012087
:108B30002DE9F04780462B48006800F114052949CB
:108B400009688889FDF737FC0521B1EB203F46DA3B
:108B5000244909688889FDF72EFC0521C1EB2030E6
:108B60004FF6FF7101EA8006002436E015F8049004
:108B7000B9F1000F06D0B9F1010F05D0B9F1020F1C
:108B800021D104E0BDE8F087601C84B224E0601CC1
:108B9000285C042802D1201DB04200DDF2E7E01C71
:108BA000295CA01C285C41EA002740F2B4508742AF
:108BB00000DC17B940F2B45000E03846A8F836009F
:108BC000201D84B208E0601C285C00B9DAE7601C54
:108BD000285C204484B200BF00BFB442C6DB00BFA3
:108BE000D0E70000D000002010B50446207EF0B190
:108BF000207E0A281BD0207E012818D0A06F20B12B
:108C0000A06FFEF7E1FA0020A067606F01F097F90E
:108C100000206067401EA086E06E01F090F9206F92
:108C200001F08DF90020E0662067A4F86A0010BD0D
:108C300070B505460C4600BF2868A04203D12868DD
:108C4000C068286017E01E49286808600EE01C48CC
:108C50000068C068A04204D11949E0680968C8608A
:108C600008E017480068C0681549086014480068A3
:108C70000028ECD100BF0020E06000BF2046FFF7D5
:108C8000B3FF207E0A280DD0207E01280AD0A07FC5
:108C900000F0010030B1A07F40F00200A077204634
:108CA000FFF7BAFD207E012805D000BF00BF00BF3E
:108CB00000BF00BF00BF0020207600BF00BF70BD16
:108CC000C40000202DE9FC4104464FF000080026B6
:108CD000FE48007800F0040070B3207E022807D11F
:108CE000FB49206D0968884211D14FF001080EE060
:108CF000F849A06A0968081A09D4A18DA06A084435
:108D0000F4490968081A002801DC4FF00108B8F19D
:108D1000000F0FD000BF00BFEF48007840F0080000
:108D2000ED490870A07F20F00100A0776FF00A00E5
:108D3000BDE8FC810020FBE7E448007800F0020079
:108D400068B1207E02280AD0207E032807D000BF09
:108D5000A07F40F00200A07700BF0020E8E7A07FDE
:108D600000F0100010B9DD4800686062002084F84F
:108D70009E002046FFF7DCFE207E801E082873D26E
:108D8000DFE800F0049BF0EFEEEDECEBCF4800786D
:108D900000F01000002877D0CC48007800F00200E6
:108DA000002871D0216FC9684868FDF7FEFA401CA1
:108DB000C7490968884267D12834E08F401CE087A2
:108DC000C4480068401C20602068A060C04800685B
:108DD0002062C3480068C0892087C1480068C089F4
:108DE0006087BC480068401EE062042004F8100C54
:108DF000E089283C211DFFF715F8E086E08E00EBA6
:108E000080004FF6FF7101EA4000A4F84E00B4F86C
:108E10004C00012802D1E08E400000E0E08EA4F872
:108E20004C0000BF00BFB4F86800401EA4F8680002
:108E3000256F28682067284601F074F8206F18B95C
:108E40004FF0FF30A08603E00020A08684F84600A3
:108E500000BFD4F8840048B100222146D4F8843001
:108E600020699847064602E0E0E10DE0002600BFD9
:108E700006F10A0010B96FF0090059E700BFA07FA2
:108E800040F00200A07717E09048007800F0100052
:108E900090B1934800680088914909684988CDE9F4
:108EA00000108C4800688F4A128881188E4B8F4AB8
:108EB0008748006800F0C2FFB9E18448007800F0FC
:108EC0001000002863D0A06C401C81490968081A72
:108ED00049D47F49206D0968081A002843DC042022
:108EE000207600BF00BF00BF606930B1002221467C
:108EF000D4E904039847064601E06FF00D0600BF71
:108F000046B106F10A0010B12046FEF781FD6FF070
:108F100009000DE7B4F84C70204600F0E1F9B4F810
:108F2000640020B1B4F86400401EA4F86400012F6E
:108F300002D1E08E400000E0E08EA4F84C006648CC
:108F4000007800F0200038B100BFA07F40F00200A0
:108F5000A07700BF0720207627E053E108E125E055
:108F6000A1E035E023E05E48006800885C490968BC
:108F70004988CDE90010574800685A4A128881187C
:108F8000594B5A4A5248006800F058FF0DE04F48CC
:108F9000007800F0020040B1A06A401E4D49096807
:108FA000884202D1204600F0C7FE40E100BF2046C3
:108FB00000F096F94848007800F0200038B100BF72
:108FC000A07F40F00200A07700BF072020762EE1AE
:108FD000204600F085F94048007800F02000E8B312
:108FE0003A48007800F01000C8B33949206D09688C
:108FF000884242D100BFA07F40F00200A07700BFAE
:109000002046FFF7F1FD00BF00BF39480068A042CD
:1090100005D137480068C0683549086018E0344811
:109020000068344908600EE032480068C068A04219
:1090300004D13049E0680968C86008E02D4800683C
:10904000C0682C4908602B4800680028ECD100BF9C
:109050000020E06000BF0120274901E016E00CE09D
:10906000087000BF0A20207600BF24480068E06036
:109070002248046001F064F914E000BFA07F40F0D2
:109080000200A07700BF082020760BE00F48007890
:1090900000F0100030B10E49206D0968884201D1FE
:1090A00006202076C3E0204600F01AF90A4800782E
:1090B00000F0200078B300BFA07F40F00200A0774E
:1090C00000BF2046FFF790FD00BF19E0E000002040
:1090D000DC000020D8000020E4000020B0000020C8
:1090E000D0000020E2000020080100200C01002038
:1090F000BC000020C4000020C8000020C0000020E8
:1091000000BF4C480068A04206D14A480068C068C9
:109110004849086019E02AE0464800684649086066
:109120000EE045480068C068A04204D14249E068AA
:109130000968C86008E040480068C0683E490860A7
:109140003D4800680028ECD100BF0020E06000BF6F
:1091500001203A49087000BF0A20207600BF384835
:109160000068E0603648046001F0EAF800BF5EE0A5
:10917000204600F0B5F83348007800F01000E0B366
:109180003149206D096888423BD12046FFF72CFD0C
:1091900000BF00BF27480068A04205D125480068ED
:1091A000C0682449086018E0224800682249086025
:1091B0000EE021480068C068A04204D11E49E06862
:1091C0000968C86008E01C480068C0681A4908605F
:1091D000194800680028ECD100BF0020E06000BF03
:1091E00001201649087000BF0A20207600BF1448ED
:1091F0000068E0601248046000E002E001F0A0F8BE
:1092000000BF14E0204600F06BF80E48007800F034
:10921000100050B10C49206D0968884205D10B48F7
:10922000007840F010000949087000E000BF00BF5E
:1092300000207DE5BC000020C4000020C800002004
:10924000C0000020E0000020DC000020E40000203E
:109250002DE9F0410446A06F477BA66F0020A06770
:1092600000BFD4F8800040B1002332462146D4F834
:1092700080C02069E047054606E0002332462146CB
:10928000184600F01FFD054600BF05BB07F0200093
:1092900020B3A08D42F23821884202D0A08D401C1C
:1092A000A08500BFD4F8800040B100231A462146B3
:1092B000D4F880C02069E047054600E0002500BFE3
:1092C00005F10A0050B96FF00900BDE8F08105F121
:1092D0000A0010B96FF00900F7E7A6670020F4E76D
:1092E0002DE9FE4F04460020009000BF00BFFE485D
:1092F000007800F0100000287ED0B4F86000A16D66
:1093000008440290F949606D0968401A15D4F7497C
:10931000606D0968884204D1F549A06D0968401A5A
:109320000BD4F349A06D0968884231D1F148006837
:10933000C089B4F8601088422ADDEE480068C08910
:10934000A4F86000B4F86200EA490968C989884253
:1093500004DAE8480068C089A4F86200E3480068BD
:109360006065E3480068A065B4F8600048B994F807
:109370009D0068B9002084F89C00012084F89D00BD
:1093800006E094F89D00002802DD002084F89D008E
:10939000D749A06C0968081A002848DC0020A4F806
:1093A0006400D548008840BBB4F86010A06D01444B
:1093B0000298814235D1B4F93400002831DBCC4920
:1093C000A06C096888422CD10120009094F84700D5
:1093D000401CC0B294F84710884204DD94F847005E
:1093E000401C84F8470094F84700032812DDB4F8C5
:1093F0004C00E18E084401E04AE10AE080B2B4F892
:109400004C1088420DDDB4F84C00E18E0844A4F8FD
:109410004C0006E094F84700032802D1204600F0F3
:10942000B8FC0098002801D184F84700ADE0A06C9A
:10943000401CAF490968081A7ED4AD49206D0968FF
:10944000081A002878DCA07F00F0040038B1A07F63
:1094500020F00400A077B4F84E00A4F84C000020DF
:109460002834A077608BB4F9181000EBE10000B24B
:10947000A083208C9E490988081AA087E08FA18FBD
:109480000844E0870020E07799480068206214F8DB
:10949000100C283C042824DBB4F84C00B4F84E101F
:1094A00088420FDAB4F84C00E18E084480B2B4F878
:1094B0004C10884215DDB4F84C00E18E0844A4F845
:1094C0004C000EE034F8361F4943E28A91FBF2F17A
:1094D000114488B2E18A363C814201DAA4F84C009A
:1094E00000BF26E0256F206F0068206700BF686816
:1094F000FDF7B8FD00BFB4F8640058B1E968888989
:10950000FCF759FF00F0010020B1B4F86400401EE0
:10951000A4F864006868FDF7A5FD34F8681F081A10
:109520002080284600F0FEFC34F8680908B100BF2E
:1095300000BF206FD8B100E024E0216FC9684868FF
:10954000FCF733FF8346216FC9688889FCF733FF36
:1095500000F0030008B1012000E00020216F09891C
:109560000844584462490968401A0028BADD206F4F
:1095700018B94FF0FF30A08601E00020A08600203F
:10958000E07702E00020A4F864002BE0E56EE06ED6
:109590000068E066E06E10B90020A4F86A0000BF21
:1095A0006868FDF75FFD00BFB4F8640058B1E96872
:1095B0008889FCF700FF00F0010020B1B4F86400D6
:1095C000401EA4F864006868FDF74CFD34F8681F7D
:1095D000081A2080284600F0A5FC34F8680908B174
:1095E00000BF00BFE06EF0B1E16EC9684868FCF7EB
:1095F000DCFE8346E16EC9688889FCF7DCFE00F07A
:10960000030008B1012000E00020E16E0989084450
:10961000584437490968081A05D43549206D096846
:10962000081A0028B2DDA06B90B33149E06B0968DD
:10963000401A2DD534F8380F30490988081A0FFA26
:1096400080FAB4F90800AAEBE0000FFA80FA20894A
:10965000504400B22081383CBAF1000F03DACAF15D
:1096600000000FFA80FA3834B4F90A00AAEBA0001F
:109670000FFA80FA6089504400B260816089B4F9C1
:10968000081000EBE10000B2A081002044F8380986
:109690001948008800286EDD207E07286BDA134801
:1096A000A16A0068401C081A66D41048A16A0068C4
:1096B000114A12881044401E081A00285CDC0B492D
:1096C000A06A0968A0EB01090D48D0F8048000BF2A
:1096D00000BF00BF00BF40684089484531DA00BF85
:1096E00000BF074840680DE0E0000020D8000020DF
:1096F000DC000020D0000020E2000020B0000020AC
:10970000240301200089A0EB090080B201900BE046
:10971000B8F80A00A9EB00090198A8F80800002091
:10972000A8F80A00D8F80080B8F80A004845EFDB2E
:10973000C9F1000001B24046FDF7ABFD58B100BFD2
:1097400009E0F8494868C9F1000109B2FDF7A1FD37
:1097500008B100BF00BFF3480089218DF24A12888A
:10976000891A401AEF490881EF49A06A0860ED495B
:10977000C96848600BE089E2EB49A06A0968081AE9
:1097800005D500BFA07F40F00200A07700BFE649EA
:10979000A06A0968081A6FD4A18DA06A0844401E07
:1097A000E1490968081A002866DCDF49A06A0968EF
:1097B00088426FD1DB49C9688889FCF7FCFD00F05D
:1097C000030008B1012000E00020D64909890844BF
:1097D000D6490880A08D0988884241DAD149C968F4
:1097E0008889FCF7E8FD00F0010098B1CD49C9680F
:1097F0008889FCF7E0FD00F03E0B5846FCF7BBFD06
:10980000C849C96889894CF2FF0211400843C5491B
:10981000C9688881A08DC3490881C9688889FCF717
:10982000CAFD00F0020020B1BE480089401EBD49BB
:109830000881BC4A11895068FDF78EFDB949C96895
:109840008889FCF7B8FD00F0030008B1012000E0B2
:109850000020B44909890844B449088000BF00BF0A
:10986000606F002815D0AF49C9688889FCF7A3FD4F
:1098700000F0010078B109E004E2D4F874B0606F40
:1098800000686067584600F04DFB00BF606F00281D
:10989000F3D172E00DE1656F2DE0E9688889FCF78E
:1098A0008AFD00F0010008B39E49C9688889FCF769
:1098B00082FD00F00200C8B90120FCF75CFD994967
:1098C000C968898908439749C96888819549C968E1
:1098D0008889FCF770FD00F0030008B1012000E06A
:1098E0000020904909890844904908802F462D6836
:1098F000384600F017FB55B1E868406829890144F3
:1099000089480068894A12881044401AC5D59DB319
:1099100085480068854909880844E9684968401A0B
:10992000002829DDE86880887F490988401A7D4938
:109930000881C9688889FCF73EFD00F0020020B16B
:1099400078480089401E77490881764A1189506815
:10995000FDF702FD7349C9688889FCF72CFD00F00A
:10996000030008B1012000E000206E490989084485
:109970006E49088000BF00BF65676B4800686B498F
:1099800009880844A06200BF00BFA08D674909880C
:10999000401AA085204600F057FD624840680089C3
:1099A000002806DD5F4840686149086000205D4985
:1099B00048605C49C9688889FCF7FDFC00F001003B
:1099C00028B15C48007840F020005A49087055E002
:1099D000666F606FC068406853490860F1688889A5
:1099E000FCF7E9FC00F0030008B1012000E00020D2
:1099F00031890844A16A0844A06200BFF1688889DF
:109A0000FCF7D9FC00BFF1688889FCF7D4FC00F0B2
:109A1000030008B1012000E0002031890844A18D35
:109A2000081AA085204600F00FFD70680089002804
:109A30000DDD3F48006828B13D4871680068FDF7BA
:109A4000F5FA02E03A497068086000207060F16839
:109A50008889FCF7B0FC00F0010050B1354800786F
:109A600040F0200033490870207E042801D10720EF
:109A7000207630686067304600F054FA606F28B195
:109A8000606FC0684068A16A8842A1D000BFA07F13
:109A900000F0010040B1A07F20F00100A077A07F7E
:109AA00040F00200A07703E0A07F40F00100A07723
:109AB00000E1204600F04FFA606F20B9194800F02D
:109AC00005FA6067F6E00027656FD7E0E868406850
:109AD00015490968884213D11248008929898842AA
:109AE0000DDD104800F0F2F906463EB10FB13E60C0
:109AF00000E0666729463046FEF746FEC1E0C0E05A
:109B0000D7B9E868406808490968081A41D5054886
:109B100000F0DCF9064626B1666729463046FEF7B6
:109B200033FEAEE024030120D8000020E200002034
:109B3000E8000020E4000020F8684068401C5E490E
:109B40000968081A25D4E8684068401E5A4909681F
:109B5000081A00281DDC594800F0B8F90646BEB1C5
:109B6000F86840683989084453490968401A002850
:109B700009DDF868808850490988081A38813989D0
:109B80007868FDF7E9FB3E6029463046FEF7FCFDAC
:109B900077E02868E8BBE868406847490968081A20
:109BA000002869DDE9688889FCF705FC00F0010000
:109BB00000B166E0414800F089F92860286848B3A0
:109BC000E8684068298908443B490968401A002828
:109BD00009DDE868808838490988081A28812989B8
:109BE0006868FDF7B9FBA18DA06A0144344800887C
:109BF000314A1268104481423DD22968C968888977
:109C0000FCF7D9FB00F00100B0B12968C968888968
:109C100001E031E02FE0FCF7CEFB00F03E0B5846B0
:109C2000FCF7A9FB2968C96889894CF2FF02114039
:109C300008432968C9688881208DA18D08441E4980
:109C40000988401A296808812A6811895068FDF737
:109C500083FB2968C9688889FCF7ADFB00F0030025
:109C600008B1012000E0002029680989084414494E
:109C7000088000BF00BF04E02F462D68002D7FF450
:109C800025AF17E0204600F066F913E00A49A06A04
:109C90000968081A08D4A18DA06A0844401E064924
:109CA0000968081A002805DD00BFA07F40F0020007
:109CB000A07700BFBDE8FE8FD8000020240301205C
:109CC000E20000202DE9F04107460D4614461E46ED
:109CD0003CB12189284600F00CF82046FDF774FAC3
:109CE00005E026B92846FDF731FFBDE8F0810020E8
:109CF000FBE770B504460E4600BF00BF00BF00BFC3
:109D0000A08D3044A085A08D42F23821884201DD2B
:109D10000846A085204600F097FB054640F68E00D9
:109D2000854208DB00BFA07F40F00200A07700BFA3
:109D30002046FEF771FD70BD2DE9F0410446206F0D
:109D400008B9BDE8F081256F2868206704F16C062A
:109D500000E03668306858B13168C9684868FCF777
:109D600024FB0746E9684868FCF71FFB381AF0D463
:109D7000306828603560286810B90020A4F86A00AF
:109D800094F84600401C84F846000020A06300BF01
:109D9000D7E710B50446206F90B3A07F00F0040011
:109DA00070BB2046FFF7C8FFB4F84C00B4F8601051
:109DB000884207DDB4F8600000EBD0714910A4F8C8
:109DC0004E1006E0B4F84C0000EBD0714910A4F836
:109DD0004E10B4F84E00E18E4900884204DAE08E5D
:109DE0004004000CA4F84E00B4F84E00E18E0322AB
:109DF00002FB0100A4F84C00A07F40F00400A07713
:109E000010BD70B50446206F00B970BD256F00E02D
:109E10002D6828680028FBD1E06E2860206FE0667E
:109E20000020206794F84600401C84F8460000207B
:109E3000A0632046FEF7F0FC00BFE6E72DE9FC5FDB
:109E400081460E4617469846DDE90CAB00221421E8
:109E50000120FCF7FBFF05460DB9BDE8FC9F00BFE4
:109E600000BF6C685046FCF786FA20805846FCF725
:109E700082FA60804846FCF771FA60603046FCF771
:109E80006DFAA06045F21400FCF775FAA08143F664
:109E90002200E0810020208260820B48B0F8780028
:109EA000401C0949A1F8780006200021FF23424602
:109EB000CDE9001039462846FCF7A2F82846FDF700
:109EC00083F900BFC9E700000002012070B5054614
:109ED00040F29D4208A10420FCF764FD04460CB941
:109EE000002070BD95E80F0084E80F006068FDF762
:109EF0006FFA2046F5E700002E2E5C5372635C5526
:109F000073725C4472697665725C557044726976EE
:109F100065725C6C7769705C636F72655C746370AA
:109F20002E63000010B5044644B1606810B160684B
:109F3000FDF74AF921460420FCF7AEFC10BD70B5D0
:109F4000044605E025682046FFF7ECFF2C4600BFDD
:109F5000002CF7D170BD2DE9FC4104460027206D8F
:109F6000FCF7FCF980464346002239462046FEF7BE
:109F700033FD054615B9B81EBDE8FC816E68A07FAB
:109F800020F00300A0770621607ACDE90001A37AD2
:109F9000221D21462846FCF733F82846FDF714F920
:109FA0000020E9E770B50446E06ED8B1E56E00E048
:109FB0002D6828680028FBD1E9688889FCF7FBF93F
:109FC00000F0070068B90120FCF7D5F9E968898934
:109FD0000843E9688881A07F40F02000A077002036
:109FE00070BD00BF01212046FDF734FFF8E70000F7
:109FF0002DE9FE4F00200290CA480068401CC94964
:10A000000860C9480078401CC749087000BF002597
:10A01000C648046858E100BF00BF00BF00BF00BFD2
:10A0200000BF94F82100C0490978884201D1E46852
:10A030004AE1BD48007884F821000026B146207E20
:10A04000022806D194F84600062802D1701CC6B238
:10A050006BE094F846000C2802D1701CC6B264E094
:10A0600094F89D0000281BDD14F89C0F401C207004
:10A07000217860789C3C401EAD4A105C814254DBE4
:10A08000002084F89C0094F89D00072804D294F8DE
:10A090009D00401C84F89D00204600F0FDF944E03E
:10A0A000B4F93400002803DBA08E401C00B2A08667
:10A0B000206FD0B3B4F93400B4F94410884234DBD3
:10A0C000207E02280CD040346088B4F9001000EBE8
:10A0D000E100A179974A515C884000B2A080403CE1
:10A0E0000020A086B4F84C00B4F86010884202DA70
:10A0F000B4F84C0001E0B4F8600082464FEA6A0010
:10A10000A4F84E00B4F84E00E18EB0EB410F06DA31
:10A11000E08E4FF6FF7101EA4000A4F84E00E08E99
:10A12000A4F84C002046FFF76CFE207E06280BD1D9
:10A13000A07F00F0100038B17A49606A0968081AF7
:10A14000282801D9701CC6B2207A00F00800A8B3F4
:10A15000207E042802D0207E07282FD12434D4E981
:10A160001C21E06E01FB02004FF4FA71B0FBF1F02C
:10A1700054F824196B4A1268511A884206D2701C8E
:10A18000C6B209F1010000F0FF0917E094F89E1033
:10A19000D4E9240201FB02004FF4FA71B0FBF1F0A4
:10A1A000604A616A1268511A884207D22046FEF757
:10A1B000C7F994F89E00401C84F89E00606F78B147
:10A1C0005849606A0968081AB4F9441001EB410162
:10A1D000B0EB410F04D3606FFFF7B1FE0020606762
:10A1E000207E032807D14F49606A0968081A282889
:10A1F00001D9701CC6B2207E092807D14949606A7E
:10A200000968081AF02801D9701CC6B2A6B3204606
:10A21000FEF7EAFC25B100BF00BFE068E86004E09B
:10A2200000BF00BF4149E0680860B9F1000F09D0E4
:10A23000A08B618BCDE90010231D2246A16A206D01
:10A24000FFF7FCFDD4F88C80D4F810B02746E46802
:10A2500039460220FCF720FB00203749087000BF78
:10A26000B8F1000F03D06FF009015846C04700BF96
:10A270003148007808B1CAE600E024E02546E468E9
:10A28000E87F401CE877E87F95F8201088421ADBC9
:10A290000020E8772849087000BFD5F8880030B161
:10A2A0002946D5F8882028699047029001E00020CF
:10A2B000029000BF2048007800B1A8E6029810B9CB
:10A2C0002846FEF7A9FA00BF002C7FF4A4AE0025B3
:10A2D0001A48046822E000BF00BF00261149606AE6
:10A2E0000968081AF02801D9701CC6B2A6B1204628
:10A2F000FEF77AFC25B100BF00BFE068E86004E02B
:10A3000000BF00BF0D49E06808602746E468394691
:10A310000220FCF7C1FA01E02546E468002CDAD1FE
:10A32000BDE8FE8FB0000020CA000020BC00002065
:10A33000E1B60000D4B60000C8000020C000002034
:10A3400010B50948006868B90848006810B908489D
:10A35000006838B101200449086000220549FA204C
:10A36000FDF714FA10BD0000F4000020BC0000202E
:10A37000C0000020C1A600001CB50446214800789A
:10A3800000F0040008B100201CBD1E48007800F059
:10A39000020008B31C49A06A0968081A24D4A18DD8
:10A3A000A06A084418490968081A00281CDC1748E4
:10A3B00000680088154909684988CDE900101248ED
:10A3C0000068134A12888118124B134A1348006818
:10A3D000FFF734FD0020D7E70A48007800F00100BD
:10A3E00010B10F480068606209480088002807DD46
:10A3F000A07F40F00200A0772046FEF70DFAC3E7E9
:10A400000020C1E7E0000020D8000020D00000209C
:10A41000E2000020080100200C010020DC000020E8
:10A42000B000002010B5FDF7BFFD06480078401CC5
:10A43000C0B20449087000F0010008B1FFF7D8FD70
:10A4400010BD0000C900002010B501468B8D886A40
:10A45000C218C88E41F21C140B6BA04201DD2046CD
:10A4600000E0C88E1844101A04D4888DC885086B83
:10A47000101A10BD0B6B886AC01A002802DD00207C
:10A48000C88506E08C6A0B6B181B00BF00BFC8852F
:10A4900000BF0020EDE700002DE9FC4705462C6FCA
:10A4A00004B9EC6E0CB9BDE8FC87E1688889FBF75C
:10A4B00082FF00F0010018B1208908B9012000E0F6
:10A4C00000208046B8F1000F01D1012000E00020FB
:10A4D0008146E06843684A4600212846FEF77CFA38
:10A4E000064606B9DFE77768B8F1000F09D01120FA
:10A4F000FBF741FFB9894CF2FF0211400843B881D4
:10A500000DE0706800F1140A616809892289891ACE
:10A510008BB2012251466068FCF70DFE00BF0B486C
:10A52000B0F87800401C0949A1F878000620002105
:10A53000CDE90010AB7A2A1D29463046FBF760FDB5
:10A540003046FCF741FE00BFADE7000000020120ED
:10A550002DE9F04105460E4617461548FDF7A0F8CF
:10A56000002822D0D82213A10720FCF71BFA0446AA
:10A570001CB94FF0FF30BDE8F08105202070A560C8
:10A58000E66027B121460A48FDF766F80BE0214650
:10A590000748FDF771F830B121460720FCF77CF938
:10A5A0004FF0FF30E7E70020E5E76FF00500E2E756
:10A5B000840000202E2E5C5372635C5573725C44E1
:10A5C00072697665725C55704472697665725C6C0E
:10A5D0007769705C6170695C74637069702E630088
:10A5E00038B504460D46FBF7CCFE0D4804600D4817
:10A5F0000560C8210C48FDF709F808B100BF00BF8D
:10A6000001210A48FDF768F808B100BF00BF042027
:10A61000430200220649009006A0FDF77DF838BDF0
:10A620007C000020800000208400002088000020A2
:10A63000F9A6000074637069705F74687265616484
:10A640000000000070B505460E461148FDF728F8D9
:10A6500010B96FF0050070BDB7220EA10820FCF7FD
:10A66000A1F9044614B94FF0FF30F4E7012020703F
:10A67000A560E66021460648FCF7FEFF30B12146A2
:10A680000820FCF709F94FF0FF30E4E70020E2E78B
:10A69000840000202E2E5C5372635C5573725C4400
:10A6A00072697665725C55704472697665725C6C2D
:10A6B0007769705C6170695C74637069702E6300A7
:10A6C00010B50446FFF7AEFE0748006810B907480A
:10A6D000006828B100220649FA20FDF757F802E089
:10A6E00000200449086010BDBC000020C00000200C
:10A6F000C1A60000F400002008B53A48006820B167
:10A70000394800683749096888474FF4FA70F9F703
:10A710008FFC00213548FCF733FF61E03348FCF73C
:10A72000F5FF69463248FDF7A5F800212F48FCF7F0
:10A7300027FF0098007807284ED2DFE800F0040CCD
:10A74000232B353F4800009A9268101D009A9268AA
:10A750001168884743E00098C06890F8350000F021
:10A76000600028B1009AD2E90201FBF739F904E050
:10A77000009AD2E90201FBF73FFB08200099FCF7A1
:10A780008BF82CE0009A9268101D009A926811686C
:10A79000884724E0009B083307CBFCF7F7FF07202E
:10A7A0000099FCF779F81AE0009AD2E90301FDF765
:10A7B000AFF807200099FCF76FF810E0009AD2E993
:10A7C0000210884707200099FCF766F807E0009A16
:10A7D000D2E90210884702E000BF00BF00BF00BFFF
:10A7E0009CE700007C000020800000208800002002
:10A7F0008400002070B505462C4600BF6068B0F1AB
:10A80000005F03D30F496068884215D3298903226A
:10A810001046FCF71BFB04464CB129462046FCF7CA
:10A820002AFC06461EB12046FCF7CEFC0024284632
:10A83000FCF7CAFC204670BD2468002CDED12846F7
:10A84000F9E700000000072070B504463748FAF722
:10A850008DFA3748F6F794FE3648F6F791FE6021F8
:10A860003548F6F7B5FE062084F82E0004F12F02D5
:10A8700000213248F6F7E8FB40F2DC50A085322098
:10A8800084F83500F6F780FF122200212B48F6F7F6
:10A890002FFD0546132200212848F6F729FD05461D
:10A8A000112200212548F6F723FD054645F0030552
:10A8B0002B46112200212148F6F733FD3C231222BA
:10A8C00000211E48F6F72DFD122200211B48F6F745
:10A8D0000FFD05464FF482611848F6F71FFC002172
:10A8E0001648F6F7B5FC064631461448F6F772FCF2
:10A8F0001248F6F75AFD1148F6F741FD10490F4886
:10A90000F6F785FC3820F6F7E5FFF7F725F80D494F
:10A910002820F6F7F9F82820F5F78CFE4FF490532D
:10A92000002211460548F6F7FCFC70BD090800F04E
:10A9300005180900051409000010064000C00E406B
:10A94000C30100807961000010B5044600BF00BF5C
:10A950000A48A062742084F8360069213720015526
:10A96000074860610748A06104F12F0003490860AF
:10A970002046FFF769FF002010BD000040010020C5
:10A980002954000049AD000070B505460C46AE6A7A
:10A9900004F4803020B110480068401C0E49086063
:10A9A00004F4004020B10D480068401C0B490860C9
:10A9B00004F0004010B1284600F012F804F0010045
:10A9C00010B1304600F068F804F4E07010B1284689
:10A9D00000F0A6F870BD00004C01002050010020DE
:10A9E000FEB50546122200212748F6F781FC0646EF
:10A9F000102200212448F6F77BFC044601220021A6
:10AA00002148F6F775FC074600BF06F4005098B1E0
:10AA100004F0010040B101201C49087001222946C0
:10AA20001B48FFF795FD07E0002018490870012238
:10AA300029461848FFF78CFD06F4A05018B36B4662
:10AA400001AA02A91048F6F72FFB04F0020020B17A
:10AA5000029820F48040029003E0029840F4804085
:10AA6000029004F0040020B1029840F400600290CB
:10AA700003E0029820F4006002900348DDE9003210
:10AA80000299F6F731FBFEBD00C00E4054010020D4
:10AA9000B76D00008D6D000070B505466C6800262E
:10AAA00039E0A16801EBC101206850F8210000F0F5
:10AAB000004000B132E0A16801EBC101206800EB69
:10AAC0008100006AE0B1A16801EBC101206800EBE0
:10AAD000810090F8200000F0010040B9A26802EB6C
:10AAE000C202216801EB8201086AFCF76DFB0020BD
:10AAF000A26802EBC202216801EB8201086200E059
:10AB00000CE0A068401CA060D4E90110884201D18B
:10AB10000020A060761C6068B042C2D800BF70BD43
:10AB20002DE9F0410546AE6AB468A06810B1A0688E
:10AB3000401E01E06068401E0746FAE0A16801EB94
:10AB4000C101206800EB8100006A002870D0A16874
:10AB500001EBC101206850F8210000F0004000B175
:10AB6000EBE0A16801EBC101206850F8210000F47E
:10AB70008070F8B1A16801EBC101206850F8210094
:10AB8000C0F30D40A26802EBC202216801EB820112
:10AB9000096A4881A16801EBC101206800EB8100CE
:10ABA000006A4089A26802EBC202216801EB8201BF
:10ABB000096A08816248006898B1A26802EBC20283
:10ABC000206800EB8200016A5D480068FCF72EFAFD
:10ABD0005B480068A26802EBC202216801EB8201B7
:10ABE0000862A16801EBC101206800EB8100006AE6
:10ABF00053490860A16801EBC101206850F82100A9
:10AC000000F48070A0B1A16801EBC101206850F888
:10AC1000210000F4004060B149480068FCF7D4FA14
:10AC20004848C088401C4749C88000204449086003
:10AC30001AE044484088401C424948802946404820
:10AC40000068FFF7FFFC60B13D480068FCF7BCFA04
:10AC50003C488089401C3B4988810846C088401C8C
:10AC6000C880002036490860032240F2EC511046AB
:10AC7000FCF7ECF8A26802EBC202216801EB82014A
:10AC800008624FF48040A26802EBC202216801EB27
:10AC900082014860A16801EBC101206800EB8100DE
:10ACA000006A70B3A16801EBC101206800EB81006C
:10ACB000006A4068A26802EBC202216801EB8201CF
:10ACC0008860A16801EBC101206800EB8100406849
:10ACD000A26802EBC202216801EB8201096A49897C
:10ACE0000843A26802EBC202216801EB82014860BE
:10ACF0004FF00040A26802EBC202216841F8220036
:10AD00000EE0FFE70020A26802EBC202216801EB1F
:10AD1000820188600B488089401C0A4988810CE0C8
:10AD2000A068401CA060D4E90110884201D1002035
:10AD3000A060A068B8427FF401AF00BFBDE8F08119
:10AD400058010020000201202DE9F84F81460E46EF
:10AD500000200090FCF710FC00903046FCF738FB18
:10AD60003046FFF747FD06465EB94E488089401CD5
:10AD70004C4988810098FCF735FC4FF0FF30BDE866
:10AD8000F88FD9F82840606800686168C96801EBED
:10AD9000C10100EB8105286A68B13046FCF714FA5E
:10ADA00040488089401C3F4988810098FCF71AFC84
:10ADB0004FF0FF30E3E73046FCF754F90746606890
:10ADC00080686168C968884205D960688068616880
:10ADD000C968401A06E06068C068C0F11800616880
:10ADE000896808448346BB450DD23046FCF7ECF930
:10ADF0002C488089401C2B4988810098FCF7F2FB85
:10AE00004FF0FF30BBE74FF0010A4FF08050286051
:10AE1000B04638E0606800686168C96801EBC1014C
:10AE200000EB8105B8F80A006860D8F80400A86053
:10AE3000BAF1000F05D04FF0000A4FF080502860A3
:10AE400001E000202860286840F4500028607F1E40
:10AE5000D8F800806068C068401C6168C86060689D
:10AE6000C068182802D100206168C8602FB928681E
:10AE700040F0C04028602E6201E0701C2862286803
:10AE800040F000402860002FC4D10748F6F789FA47
:10AE900004480088401C034908800098FCF7A2FB86
:10AEA00000206CE70002012000C00E407047000047
:10AEB0002DE9FF5F05460E467B48B0F86200401C56
:10AEC00081B27948A0F86210D5F804B029899BF8BE
:10AED000000000F00F00082202EB8000814208DB36
:10AEE0009BF800000007800E41422846FCF7D1F98C
:10AEF00090B16D48B0F86A00401C81B26A48A0F871
:10AF00006A10B0F86600401C81B26748A0F866106D
:10AF10002846FCF759F9C4E0D5F80490634908685D
:10AF20003146FAF742FF8046B9F80000FBF743FAD2
:10AF30000390B9F80200FBF73EFA029000270020C8
:10AF4000019082465A4804684CE000200190618AD2
:10AF50000298814223D1B8F1000F02D1ACB1206830
:10AF600098B152492068096888420ED0B8F1000FA4
:10AF700015D054B1206840B12168B06801404B48F9
:10AF80000068B2681040814209D101200190BAF1F5
:10AF9000000F04D1207C00F0040000B9A246019803
:10AFA000F0B1A18A039881421AD1201D30B16068A6
:10AFB00020B1404960680968884211D13FB1E0681A
:10AFC000F8603B480068E0603948046007E03648B4
:10AFD000B0F87600401C81B23348A0F8761003E048
:10AFE0002746E468002CB0D100BF04B9544624B908
:10AFF0002E497068096888424FD16FF007012846D2
:10B00000FCF747F968B100BF00BF2748B0F86600F9
:10B01000401C81B22448A0F866102846FCF7D4F8FA
:10B020003FE074B1A06940B103980090214B2A46DB
:10B030002146D4E906C0E04732E02846FCF7C4F8D0
:10B040002FE0B8F1000F15D11848007800F0F0009B
:10B05000E0280FD09BF8000000F00F00082202EB60
:10B0600080012846FCF715F900BF00BF03212846E0
:10B07000FAF72AFD0C48B0F87000401C81B20A486B
:10B08000A0F87010B0F86600401C81B20648A0F825
:10B0900066102846FCF798F802E02846FCF794F87A
:10B0A00000BFBDE8FF9F0000000201200C0100204E
:10B0B000FC000020080100200090D0030C000000DC
:10B0C00000EA32060000000080D1F0080400000011
:10B0D000004000401000000000800540100000000B
:10B0E00000500040110000000090054011000000D9
:10B0F000006000401200000000A0054012000000A7
:10B10000007000401300000000B005401300000074
:10B11000004002401400000000C005401400000080
:10B12000005002402E00000000D005402E0000001C
:10B13000006002402F00000000E005402F000000EA
:10B14000007002403000000000F0054030000000B8
:10B1500000D003404600000000000640460000000A
:10B160000010064047000000002006404800000094
:10B17000003006407F0000000040064080000000D4
:10B180000050064084000000006006408C00000073
:10B19000004000401000000000800540100000004A
:10B1A0000050004011000000009005401100000018
:10B1B000006000401200000000A0054012000000E6
:10B1C000007000401300000000B0054013000000B4
:10B1D000004002401400000000C0054014000000C0
:10B1E000005002402E00000000D005402E0000005C
:10B1F000006002402F00000000E005402F0000002A
:10B20000007002403000000000F0054030000000F7
:10B2100000D003404300000000000640430000004F
:10B2200000100640440000000020064045000000D9
:10B230000030064058000000004006405900000061
:10B24000005006405C000000006006406400000002
:10B25000007006406C000000008006406D00000099
:10B26000009006407F000000004000400080054044
:10B2700000500040009005400060004000A00540E4
:10B280000070004000B005400040024000C0054092
:10B290000050024000D005400060024000E0054040
:10B2A0000070024000F0054000D00340000006405E
:10B2B0000010064000100640002006400020064016
:10B2C0000030064000300640004006400040064086
:10B2D00000500640005006400060064000600640F6
:10B2E0000070064000700640008006400080064066
:10B2F0000090064000900640000700000006000095
:10B30000000500000004000000030000000200002F
:10B3100000010000000000000000000018ED00E047
:10B320001CED00E020ED00E000E400E004E400E0BB
:10B3300008E400E00CE400E010E400E014E400E0C5
:10B3400018E400E01CE400E020E400E024E400E075
:10B3500028E400E02CE400E030E400E034E400E025
:10B3600038E400E03CE400E040E400E044E400E0D5
:10B3700048E400E04CE400E050E400E054E400E085
:10B3800058E400E05CE400E060E400E064E400E035
:10B3900068E400E06CE400E070E400E074E400E0E5
:10B3A00078E400E07CE400E080E400E084E400E095
:10B3B00088E400E000E100E004E100E008E100E0F2
:10B3C0000CE100E010E100E080E100E084E100E059
:10B3D00088E100E08CE100E090E100E000E200E0C4
:10B3E00004E200E008E200E00CE200E010E200E02D
:10B3F00080E200E084E200E088E200E08CE200E02D
:10B4000090E200E0010000007856341201003F0095
:10B4100001001800E80501000100100014000200FE
:10B420000A0001003F00010001000A0001001800AD
:10B43000F0000100040001000A00180008000100EB
:10B44000040001000100010080000100340001003F
:10B450000100800001000100010040005800E803E5
:10B4600001001A720100100001000800E803280022
:10B470008002080040006224000001000200010078
:10B4800003000100020001000400010002000100AD
:10B49000030001000200010005000100020001009C
:10B4A000030001000200010004000100020001008D
:10B4B000030001000200010006000100020001007B
:10B4C000030001000200010004000100020001006D
:10B4D000030001000200010005000100020001005C
:10B4E000030001000200010004000100020001004D
:10B4F000030001000200010007000100020001003A
:10B50000030001000200010004000100020001002C
:10B51000030001000200010005000100020001001B
:10B52000030001000200010004000100020001000C
:10B5300003000100020001000600010002000100FA
:10B5400003000100020001000400010002000100EC
:10B5500003000100020001000500010002000100DB
:10B5600003000100020001000400010002000100CC
:10B5700003000100020001001C002000A0001C00CC
:10B5800010001000300014001400100030001C06E1
:10B59000040004000700040014000A00080008006A
:10B5A00010001000300014006465746563746564F5
:10B5B000206D656D70206F766572666C6F7720699F
:10B5C0006E20706F6F6C2000000000000000000013
:10B5D000000000000000000000000000000000006B
:10B5E000000000000000000000000000000000005B
:10B5F000000000000000000000000000000000004B
:10B60000000000000000000000000000000000003A
:10B61000000000000000000000000000000000002A
:10B6200000000000000000006465746563746564D8
:10B63000206D656D7020756E646572666C6F772025
:10B64000696E20706F6F6C20000000000000000029
:10B6500000000000000000000000000000000000EA
:10B6600000000000000000000000000000000000DA
:10B6700000000000000000000000000000000000CA
:10B6800000000000000000000000000000000000BA
:10B6900000000000000000000000000000000000AA
:10B6A000000000000000000028B7000050B70000B4
:10B6B00070B7000030B700001CB7000004B70000EE
:10B6C00010B7000064B700003CB7000044B70000AA
:10B6D00058B700000102030405060707070707071C
:10B6E0000703060C18306078B8000020B400002072
:10B6F000BC000020C0000020FFFFFFFFFFFF000094
:10B700000000000046494E5F574149545F31000038
:10B7100046494E5F574149545F32000045535441FA
:10B72000424C495348454400434C4F534544000064
:10B7300053594E5F5243564400000000434C4F5350
:10B74000494E47004C4153545F41434B00000000B9
:10B750004C495354454E000054494D455F574149AB
:10B7600054000000434C4F53455F5741495400007B
:10B7700053594E5F53454E54000000009CB70000E3
:10B78000000000208C01000064040000D0B700001D
:10B790008C010020EC6A01001051000001AD021E76
:10B7A000C00B486E194C1AFF01131801B720B82AB4
:10B7B000012018F6182E0120081A20281A30040932
:10B7C00023773EA804E6FFFF0842018B7A0470004D
:0400000500000201F4
:00000001FF
